:100000000C94C3070C94EB070C94EB070C94EB07D0
:100010000C94EB070C94EB070C94EB070C94EB0798
:100020000C94EB070C94EB070C94EB070C94EB0788
:100030000C94EB070C94EB070C94EB070C94EB0778
:100040000C94EB070C94EB070C9452510C94EB07B7
:100050000C94A4530C94EB530C94EB070C94EB0707
:100060000C94EB070C94EB070C94A34F0C94EB0748
:10007000485454502F312E3020323030204F4B0D09
:100080000A436F6E74656E742D547970653A2074EE
:100090006578742F68746D6C0D0A507261676D61BC
:1000A0003A206E6F2D63616368650D0A0D0A004882
:1000B0005454502F312E3020323030204F4B0D0A07
:1000C000436F6E74656E742D547970653A2061705B
:1000D000706C69636174696F6E2F6A736F6E0D0A5D
:1000E000436F6E6E6E656374696F6E3A20636C6FFA
:1000F00073650D0A0D0A003C6D657461206E616DBB
:10010000653D76696577706F727420636F6E746594
:100110006E743D2277696474683D363430223E0D3A
:100120000A00485454502F312E302034303120559D
:100130006E617574686F72697A65640D0A436F6EDB
:1001400074656E742D547970653A20746578742FD7
:1001500068746D6C0D0A0D0A3C68313E34303120F4
:10016000556E617574686F72697A65643C2F683189
:100170003E0077696E646F772E6C6F636174696F90
:100180006E3D222F223B3C2F7363726970743E0ACE
:10019000006376007670006D70006470006370001C
:1001A000677000766F00636F00736E007073007687
:1001B00073006373007672006372006A6F006A6E88
:1001C000006A70006A63007375006375002446005E
:1001D00024440024440024460024463C6D65746198
:1001E00020687474702D65717569763D227265663C
:1001F000726573682220636F6E74656E743D223180
:100200003B2075726C3D2F223E0024463C73637286
:100210006970743E616C65727428224F7074696FE6
:100220006E732076616C7565732073617665642EDC
:1002300022293B24460024463C7363726970743E55
:10024000616C65727428224E6577207061737377D4
:100250006F726473206D757374206D6174636821AF
:1002600022293B77696E646F772E6C6F63617469C6
:100270006F6E3D222F766F223B3C2F736372697045
:10028000743E0A0024463C7363726970743E616C6C
:1002900065727428224E65772070617373776F7270
:1002A00064207365742E22293B24460024463C7347
:1002B00063726970743E616C657274282256616C59
:1002C000756573206F7574206F6620626F756E643C
:1002D0002122293B77696E646F772E6C6F6361749E
:1002E000696F6E3D222F766F223B3C2F73637269DC
:1002F00070743E0A0024463C7363726970743E61F8
:100300006C65727428225363726970742075726C04
:100310002073617665642E22293B24460024463CE6
:100320007363726970743E2446005265626F6F7425
:10033000696E672E2E2E0024463C6D657461206820
:100340007474702D65717569763D2272656672658B
:1003500073682220636F6E74656E743D2224443B83
:100360002075726C3D2F223E003C7363726970747D
:10037000207372633D2224452F766965776F702E56
:100380006A73223E3C2F7363726970743E0A003CAC
:100390002F7363726970743E0A00305D3B76617240
:1003A000206E6F7074733D24442C6C6F633D222467
:1003B00045222C646576743D244C2C747A3D24448B
:1003C0003B00222446222C24442C24442C24442C5C
:1003D000003C7363726970743E766172206F707452
:1003E000733D5B0024462446002264756D6D7922BE
:1003F0003A307D00222446223A24442C007B0024FB
:1004000046003C736372697074207372633D2224EA
:10041000452F686F6D652E6A73223E3C2F736372A1
:100420006970743E0A000A766172206C72756E3DC6
:100430005B24442C24442C24442C244C5D3C2F73FA
:1004400063726970743E0A005B302C305D5D3B0A5C
:1004500076617220656E3D24442C72643D24442CE8
:1004600072733D24442C6D6D3D24442C726473746E
:100470003D244C2C6D61733D24442C7572733D24D6
:10048000442C776C3D24442C697061733D24442CCA
:100490006C6F633D222445223B005B24442C244C9A
:1004A0005D2C00305D3B7661722070733D5B0024F3
:1004B000442C00766172206E6272643D24442C7478
:1004C0007A3D24442C73626974733D5B00766172DB
:1004D000207665723D24442C646576743D244C3B43
:1004E0000A00244624463C7363726970743E0030EF
:1004F0002C305D7D0024442C244C2C00305D2C22BB
:100500007073223A5B0024442C007B22646576746D
:10051000223A244C2C226E627264223A24442C2209
:10052000656E223A24442C227264223A24442C22FE
:100530007273223A24442C226D6D223A24442C22D8
:1005400072647374223A244C2C226C6F63223A2218
:100550002445222C227362697473223A5B0024467C
:100560000077696E646F772E6C6F636174696F6E6C
:100570003D222F7670223B3C2F7363726970743E6C
:100580000A00616C657274282250726F6772616D27
:10059000202444206D6F64696669656422293B00EC
:1005A000616C65727428224E65772070726F677275
:1005B000616D2061646465642E22293B0024463C01
:1005C0007363726970743E003C7363726970742067
:1005D0007372633D2224452F706C6F7470726F6765
:1005E0002E6A73223E3C2F7363726970743E0A0058
:1005F000305D3B0024442C00766172206D61736F86
:10060000703D5B00766172207365713D24442C6DF2
:1006100061733D24442C776C3D24442C7364743DF9
:1006200024442C6D746F6E3D24442C6D746F66668B
:100630003D24442C6465766461793D24442C6465D2
:10064000766D696E3D24442C64643D24442C6D6DAC
:100650003D24442C79793D24443B0024463C73637B
:10066000726970743E0024463C7363726970743E14
:1006700077696E646F772E6C6F636174696F6E3D1E
:10068000222F7670223B3C2F7363726970743E0A8E
:10069000003C2F7363726970743E0A3C7363726925
:1006A0007074207372633D2224452F6D6F647072E5
:1006B0006F672E6A73223E3C2F7363726970743EBB
:1006C0000A005D3B002C2444007661722070726F3A
:1006D000673D5B24442C24442C24442C24442C24A7
:1006E000442C24442C244400766172206E626F6195
:1006F0007264733D24442C7069643D24442C6970F9
:1007000061733D24443B00244624463C7363726974
:1007100070743E003C736372697074207372633D41
:100720002224452F7669657770726F672E6A73226F
:100730003E3C2F7363726970743E0A00244624465F
:100740003C7363726970743E0024463C7363726943
:1007500070743E2446003C73637269707420737237
:10076000633D2224452F76696577726F2E6A732266
:100770003E3C2F7363726970743E0A00305D3B3CEF
:100780002F7363726970743E0A0024442C007661F2
:1007900072206E626F617264733D24442C6D6173CC
:1007A0003D24442C697061733D24442C6475723D72
:1007B0005B00244624463C7363726970743E005BA0
:1007C000302C302C302C302C302C302C302C305D18
:1007D0005D7D005D2C002C2444005B24442C2444CB
:1007E0002C24442C24442C24442C24442C24440025
:1007F0007B226E70726F6773223A24442C226E62E1
:100800006F61726473223A24442C226D6E70223A16
:1008100024442C227064223A5B002446003C687217
:10082000202F3E3C666F726D206E616D653D6F6678
:1008300020616374696F6E3D6375206D6574686FC8
:10084000643D6765743E3C703E3C623E4A61766141
:100850007363726970742055524C3A3C2F623E208B
:100860003C696E70757420747970653D7465787438
:100870002073697A653D3332206D61786C656E67EF
:1008800074683D3132372076616C75653D222445B0
:1008900022206E616D653D6A73703E3C2F703E3C58
:1008A000703E5365742055524C2077686572652000
:1008B0004A61766173637269707473206172652036
:1008C00073746F7265642E2044656661756C742064
:1008D000697320687474703A2F2F72617973686F2E
:1008E0006262792E6E65742F736372697074732FF0
:1008F0006A6176612F737663322E302E333C6272DA
:10090000202F3E4966206C6F63616C206F6E2075EE
:10091000534420636172642C20757365202E202857
:10092000692E652E20646F74293C2F703E3C703E0A
:100930003C623E50617373776F72643A3C2F623E43
:100940003C696E70757420747970653D7061737365
:10095000776F72642073697A653D3130206E616D06
:10096000653D70773E3C696E707574207479706572
:100970003D7375626D69743E3C2F703E3C68722019
:100980002F3E3C2F666F726D3E002446003C2F7355
:1009900063726970743E0A005D3B002C2444007051
:1009A000645B24445D3D5B24442C24442C24442C6F
:1009B00024442C24442C24442C24440076617220AA
:1009C0006E70726F67733D24442C6E626F61726447
:1009D000733D24442C697061733D24442C6D6E700A
:1009E0003D24442C70643D5B5D3B0024463C7363B6
:1009F000726970743E616C65727428224368616E1E
:100A00006765732073617665642E22293B24460056
:100A100027275D3B00272453272C00766172207323
:100A20006E616D65733D5B00305D3B3C2F7363729F
:100A30006970743E0A3C73637269707420737263E8
:100A40003D2224452F76696577736E2E6A73223EA8
:100A50003C2F7363726970743E0A0024442C007644
:100A60006172206D61736F703D5B00766172206E04
:100A7000626F617264733D24442C6D61786C656EA5
:100A80003D24442C6D61733D24442C697061733D99
:100A900024443B0024463C7363726970743E00300A
:100AA0005D2C226D61786C656E223A24447D0024B1
:100AB000442C002264756D6D79225D2C226D61736A
:100AC0006F70223A5B00222453222C007B22736E2B
:100AD000616D6573223A5B002446004E54502053EA
:100AE000796E63696E672E2E2E00436F6E6E65639E
:100AF00074696E672E2E2E00446574656374696E8A
:100B000067207553442E2E2E0066777600747A0087
:100B10006E747000646863700069703100697032CF
:100B2000006970330069703400677731006777328D
:100B30000067773300677734006870300068703181
:100B400000617200657874007365710073647400ED
:100B50006D6173006D746F6E006D746F66007572F9
:100B6000730072736F00776C007374740069706146
:100B70007300646576696400636F6E006C6974006D
:100B80006E747031006E747032006E747033006E6B
:100B9000747034007265736574004669726D7761B4
:100BA0007265207665722E0054696D65207A6F6ECD
:100BB000653A004E54502073796E633F005573655B
:100BC00020444843503F005374617469632E697038
:100BD000313A005374617469632E6970323A00537C
:100BE00074617469632E6970333A00537461746977
:100BF000632E6970343A00476174657761792E69B4
:100C000070313A00476174657761792E6970323AC4
:100C100000476174657761792E6970333A004761E6
:100C200074657761792E6970343A004854545020C5
:100C3000706F72743A00004175746F207265636F53
:100C40006E6E6563743F0023206F66206578702E9A
:100C500020626F6172643A0053657175656E7469E4
:100C6000616C206D6F64653F0053746174696F6ED1
:100C70002064656C61793A004D617374657220730C
:100C8000746174696F6E3A004D61737465722020EF
:100C90006F6E2061646A2E3A004D61737465722034
:100CA0006F66662061646A2E3A0055736520726132
:100CB000696E2073656E736F723A004E6F726D616C
:100CC0006C6C79206F70656E3F00252057617465EC
:100CD000722074696D653A0053656C66746573744F
:100CE0002074696D653A0049676E6F7265207061A6
:100CF0007373776F72643F0044657669636520495A
:100D0000443A004C434420436F6E74726173743AEA
:100D1000004C4344204261636B6C696768743A001D
:100D20004E5450207365727665722E6970313A00A8
:100D30004E5450207365727665722E6970323A0097
:100D40004E5450207365727665722E6970333A0086
:100D50004E5450207365727665722E6970343A0075
:100D6000526573657420616C6C3F004D6F6E00546A
:100D700075650057656400546875004672690053D4
:100D800061740053756E00206D696E002073656399
:100D90000025004E6F00596573002B002B00204783
:100DA0004D54003030003A002D002B000020202050
:100DB00020002D5261696E2053746F702D002D44F8
:100DC000697361626C6564212D003A0045004D43F2
:100DD0003A003A002E002D0020002020003A00208A
:100DE0000042333A686F6C6420746F2073617665DB
:100DF0000042333A73656C2042312F42323A6368C5
:100E000067003D3D536574204F7074696F6E733D8C
:100E10003D00506C6561736520576169742E2E2EFC
:100E200000526573657474696E6720454550524F72
:100E30004D0000010800060400014500008200008A
:100E400040002000504F5354202446204854545012
:100E50002F312E300D0A486F73743A2024460D0A44
:100E6000244624534163636570743A202A2F2A0D67
:100E70000A436F6E74656E742D4C656E6774683AC4
:100E80002024440D0A436F6E74656E742D5479707E
:100E9000653A206170706C69636174696F6E2F7858
:100EA0002D7777772D666F726D2D75726C656E6319
:100EB0006F6465640D0A0D0A2453004745542024CD
:100EC00046245320485454502F312E300D0A486F79
:100ED00073743A2024460D0A24460D0A0D0A004177
:100EE00063636570743A20746578742F68746D6CF0
:100EF00000E30004FA0001000000010000210024CA
:100F00000027002A0000002200250028002B0000F6
:100F10000020002300260029000202020202020231
:100F2000020404040404040404030303030303038A
:100F30000301010101010101010102040810204027
:100F400080010204081020408001020408102040A3
:100F5000808040201008040201000000010200000F
:100F6000000000000004030706000000000000006D
:100F700000000000000000000000590A60298F34C2
:100F8000FF463F4ECB5411241FBECFEFD0E1DEBF52
:100F9000CDBF13E0A0E0B1E0E6E9FFEA02C00590B2
:100FA0000D92AC35B107D9F71DE0ACE5B3E001C057
:100FB0001D92A33AB107E1F71FE0C6E8DFE004C0E5
:100FC0002297FE010E948E57CA37D107C9F70E94A7
:100FD0001B550C94C9570C940000FC0188279927D5
:100FE000E89421912032E9F3293010F02E30C8F333
:100FF0002B3241F02D3239F4689404C00E94270945
:10100000820F911D219120532A30C0F31EF4909538
:1010100081959F4F08951F93FC0199278827BC0154
:10102000E89411911032E9F3193010F01E30C8F332
:101030001B3251F01D3249F4689406C00E94120917
:10104000610F711D811D911D119110531A30B0F364
:101050003EF490958095709561957F4F8F4F9F4F8F
:101060001F910895FB01DC0102C005900D924150D3
:101070005040D8F70895FB01DC0104C08D91019028
:10108000801921F441505040C8F7881B990B0895EE
:10109000DC0101C06D9341505040E0F70895FB0121
:1010A000DC018D91019080190110D9F3990B0895FD
:1010B000FB01DC0101900D920020E1F70895FB0196
:1010C000DC014150504030F08D910190801919F4AD
:1010D0000020B9F7881B990B0895A0E0B0E0E3E782
:1010E000F8E00C949C577C01EB018A01690109C06E
:1010F000CE012196F6010995F70181937F010150F8
:10110000104001151105A1F7CDB7DEB7E8E00C944A
:10111000B857BF92CF92DF92EF92FF920F931F9337
:101120007B018C01FB010995B82EC8010196F701DE
:101130000995C82EC8010296F7010995D82EC80155
:101140000396F7010995982F6B2D7C2D8D2D1F91FE
:101150000F91FF90EF90DF90CF90BF900895A0E0A7
:10116000B0E0E5EBF8E00C949C57EC017B018A01C0
:10117000690109C0CE012196F70161917F01F60155
:1011800009950150104001151105A1F7CDB7DEB743
:10119000E8E00C94B857BF92CF92DF92EF92FF92A3
:1011A0000F931F93D52EC62EB72E79018C01642F75
:1011B000F9010995C80101966D2DF7010995C8013E
:1011C00002966C2DF7010995C80103966B2DF70166
:1011D00009951F910F91FF90EF90DF90CF90BF90F6
:1011E0000895FB019F01E8944230C4F04532B4F405
:1011F0004A3029F497FB1EF4909581959F4F642FF8
:1012000077270E944357805D8A330CF0895D819374
:10121000CB010097A1F716F45DE251931082C9014A
:101220000C945409592F482F372F262F660F771FFC
:10123000881F991F660F771F881F991F620F731FE2
:10124000841F951F660F771F881F991F08957AE0E6
:10125000979F902D879F802D910D11240895FA015D
:10126000CF93FF93EF932230CCF02532BCF4C22F02
:101270002C2F332744275527FF93EF930E946A575B
:10128000EF91FF91605D6A330CF0695D6193B90184
:10129000CA01605070408040904051F710828F9199
:1012A0009F91CF910C945409DC01FC01672F71913F
:1012B0007723E1F7329704C07C916D93708362913C
:1012C000AE17BF07C8F308959C01F999FECF32BD50
:1012D00021BDF89A80B508959C01F999FECF1FBAF7
:1012E00032BD21BD60BD0FB6F894FA9AF99A0FBECF
:1012F0000895FC01A681B7816D93B783A68381E031
:1013000090E00895CF92DF92EF92FF920F931F9398
:10131000CF93DF937B018C010894E11CF11C011D2C
:10132000111DC090FE08442361F43091FB083695EE
:10133000369536953170A8EEB7E0C8E2D7E0DD24E7
:1013400071C09091FB089695969596959170C8EE10
:10135000D7E068E277E0EC2DF0E0EE0FFF1FEE0F34
:10136000FF1FEC0FFD1F25C0288139814A815B8159
:101370002115310541055105C9F0DB01ED92FD92C2
:101380000D931C931397D801C701820F931FA41FBD
:10139000B51F88839983AA83BB83209144027C0173
:1013A0008D01E20EF11C011D111D91E024966C5F70
:1013B0007F4FCE17DF07C1F69170990F990F990FE4
:1013C0008091FB08877F892B37C04D915D916D918E
:1013D0007C911397411551056105710501F1ED2DC2
:1013E000E695E695E695F0E0E150F74F808190E0D4
:1013F0002D2D277002C0959587952A95E2F780FDDF
:101400000EC0E882F9820A831B834E0D5F1D601FA8
:10141000711F4D935D936D937C93139731E0D3943B
:1014200014962496DC1488F23170330F330F330F87
:101430008091FB08877F832B8093FB08DF91CF91FE
:101440001F910F91FF90EF90DF90CF900895A8EA41
:10145000B8E080E090E0FC01E85DF84F1082118276
:1014600012821382FC01E851F84F1082118212821D
:1014700013821D920496803C910569F7F999FECF7D
:1014800086E694E092BD81BDF89A80B580931F07EF
:101490001092200710922107109223071092220722
:1014A0001092240710922507109226071092270702
:1014B0000895109216071092150788EF92E0909306
:1014C00014078093130708959F92AF92BF92CF9213
:1014D000DF92EF92FF920F931F93CF93DF93EC0174
:1014E000962E87ED99E0BE010E94524A882309F4A6
:1014F00058C087ED99E0BE0141E00E94384BAA2414
:10150000BB24650187ED99E00E943347EC01A8E117
:10151000BAE026E330E040E050E0A20EB31EC41E65
:10152000D51EF501E25AFC4F2AEC3FEF4FEF5FEF7B
:10153000A20EB31EC41ED51E8601750107C00894F5
:10154000E11CF11C011D111D8D918193C7018A19A8
:101550009B098C179D079CF330E0E31632E0F306FD
:1015600030E0030730E0130748F0C70160E140E0D6
:101570000E94ED35AA24BB2465010AC041E09416FF
:1015800029F4C70161E140E00E94ED35570168018F
:10159000C050D24009F4B6CF87ED99E00E94F846DA
:1015A00081E0DF91CF911F910F91FF90EF90DF903D
:1015B000CF90BF90AF909F900895CF92DF92FF920F
:1015C0000F931F93CF93DF9300D000D000D0EDB7DF
:1015D000FEB7319603E117E0ADB7BEB712961C9384
:1015E0000E9311978FEF93E0938382838FEA90E0BD
:1015F000958384830E94093B0F900F90EDB7FEB74F
:10160000128301838DEF93E0948383830E94093BCF
:10161000CDECD1E0FF240F900F900F900F9094EF3E
:10162000C92E93E0D92E2C813D818881F4E1FF16EB
:1016300019F490E0CC9701C090E04DB75EB74850E8
:1016400050400FB6F8945EBF0FBE4DBFEDB7FEB76A
:101650003196ADB7BEB711960C93119712961C93A5
:10166000D382C28235832483978386830E94093B79
:10167000F3942796EDB7FEB738960FB6F894FEBFF1
:101680000FBEEDBFF2E2FF1671F600D000D0ADB78D
:10169000BEB711960C93119712961C93129789EE70
:1016A00093E014969C938E9313970E94093B0F909E
:1016B0000F900F900F9081E0DF91CF911F910F91CC
:1016C000FF90DF90CF9008950F931F9300D000D02C
:1016D00000D0EDB7FEB7319603E117E0ADB7BEB766
:1016E00012961C930E9311978AE899E09383828354
:1016F00080E790E0958384830E94093BEDB7FEB7B5
:101700003196ADB7BEB712961C930E9311978DE12B
:1017100098E09383828380E890E0958384830E949D
:10172000093B8DB79EB706960FB6F8949EBF0FBEC5
:101730008DBF81E01F910F910895CF92DF92EF92BC
:10174000FF920F931F93DF93CF9300D000D0CDB7BC
:10175000DEB70E949A517B018C016E010894C11C76
:10176000D11C0E9485420E941438C60160918001FC
:101770000E9413358823E1F0E980FA800B811C81F7
:1017800080EC98EDA4E5BCE7E80EF91E0A1F1B1FCC
:101790006091D40170E080E090E024E833E040E024
:1017A00050E00E941857E60EF71E081F191F0EC0C2
:1017B0000E949A516E197F09800B910B685B7B40E8
:1017C0008040904070F2EE24FF248701B701C801E9
:1017D0000F900F900F900F90CF91DF911F910F916D
:1017E000FF90EF90DF90CF900895EF92FF921F93BC
:1017F000DF93CF9300D000D0CDB7DEB780919802B1
:10180000898380919F028A838091A6028B83809135
:10181000AD028C8310E07E010894E11CF11C609104
:1018200080016F5F60938001C7010E9476370E943C
:101830009D0B9B01AC01611571058105910519F4A2
:101840001F5F143161F7B901CA010F900F900F901B
:101850000F90CF91DF911F91FF90EF900895CF935C
:10186000DF939C011092E206FC01A081B181C0E0EF
:10187000D0E00FC09C919D3231F09B3221F0892F36
:1018800080538A3068F4FE01EE51F94F908321961F
:101890001196F901808191810A96A817B90750F332
:1018A000CE51D94F18821196F901B183A08382EEEF
:1018B00096E00E94ED07DF91CF910895BF92CF92FD
:1018C000DF92EF92FF920F931F93CF93DF932DB789
:1018D0003EB7285030400FB6F8943EBF0FBE2DBF24
:1018E000EDB7FEB7319603E117E0ADB7BEB712967C
:1018F0001C930E93119784EE93E09383828380E789
:1019000090E09583848387EF90E0978386830E949D
:10191000093B0F900F900F900F90EDB7FEB7128319
:10192000018381ED93E0948383830E94093B2DEC36
:10193000E22E21E0F22EDD24C0E0D0E00F900F90E7
:101940000F900F90B02EC12E02EC13E05C2F6D2F84
:10195000D70116968C91169781FF33C014962D915E
:101960003C91159711964C9111978C91C43119F4B3
:1019700090E0CC9701C090E0EDB7FEB73C970FB672
:10198000F894FEBF0FBEEDBF3196ADB7BEB711964E
:10199000BC9211971296CC921383028335832483D1
:1019A0004683178291878087528763870E94093B0D
:1019B000D394EDB7FEB73C960FB6F894FEBF0FBEBA
:1019C000EDBF219627E030E0E20EF31EC232D105D2
:1019D00009F0BCCF0E946E46ADB7BEB71E970FB6DA
:1019E000F894BEBF0FBEADBFEDB7FEB7319603E1B1
:1019F00017E012961C930E9311972AE933E0338374
:101A00002283D482158220E630E0378326836087E4
:101A10007187828793878091D401848715860E947D
:101A2000093BEDB7FEB73A960FB6F894FEBF0FBE6E
:101A3000EDBF128301838FE893E0948383830E9438
:101A4000093B00D0EDB7FEB73196ADB7BEB71296E1
:101A50001C930E93119789E693E09383828380E829
:101A600090E0958384830E94093BEDB7FEB73696DC
:101A70000FB6F894FEBF0FBEEDBF81E0DF91CF91AE
:101A80001F910F91FF90EF90DF90CF90BF9008953E
:101A90004F925F926F927F928F929F92AF92BF927E
:101AA000CF92DF92EF92FF920F931F93DF93CF932A
:101AB0000F92CDB7DEB70E946E465B016C0100D07D
:101AC00000D000D0EDB7FEB7319603E117E0ADB717
:101AD000BEB712961C930E9311978EE595E09383F3
:101AE00082838FEA90E0958384830E94093BEDB75F
:101AF000FEB772970FB6F894FEBF0FBEEDBF3196DA
:101B0000ADB7BEB712961C930E9311978AE095E07D
:101B100093838283A482B582C682D7828091FD0896
:101B2000808711868091FB0881708287138680915F
:101B3000FB0886958170848715868091FB088695C1
:101B400086958170868717868091FB0882958170C3
:101B5000808B118A80910B0990910C09A0910D093D
:101B6000B0910E09828B938BA48BB58B80E690E0AD
:101B7000978B868B0E94093B90E0EDB7FEB7789675
:101B80000FB6F894FEBF0FBEEDBF780106E015E07A
:101B900023C000D000D000D0EDB7FEB73196ADB76E
:101BA000BEB71196EC9211971296FC9213830283A2
:101BB000A92FB0E0A150B74F8C91848315829983EF
:101BC0000E94093B99819F5FEDB7FEB736960FB62D
:101BD000F894FEBF0FBEEDBF8091FD08A3E16A2E11
:101BE000A7E07A2E9817A8F200D000D0ADB7BEB704
:101BF00012967C926E9211978CEF94E014969C93BF
:101C00008E9313970E94093B99240F900F900F9089
:101C10000F90C301762C892EF5EF4F2EF4E05F2E46
:101C200066C0A92DB0E0FD01E855F74F608166233D
:101C3000A9F1CD01880F991F880F991FFC01E85D5C
:101C4000F84FE080F18002811381FC01E851F84FE8
:101C5000AE14BF04C006D10648F020813181428114
:101C600053812A193B094C095D0908C02081318143
:101C7000428153812E193F09400B510BAA0FBB1F04
:101C8000AA0FBB1FA851B84F8D919D910D90BC918B
:101C9000A02D8E5F9F4FAF4FBF4F21F420E030E06B
:101CA00040E050E08DB79EB70A970FB6F8949EBFFC
:101CB0000FBE8DBFEDB7FEB73196ADB7BEB711966B
:101CC0007C92119712968C92538242826483158281
:101CD00026833783408751870E94093B9394EDB751
:101CE000FEB73A960FB6F894FEBF0FBEEDBF8091D7
:101CF000FE08981608F495CF00D000D083E197E055
:101D0000ADB7BEB712969C938E9311978FEE94E069
:101D100014969C938E9313970E94093B81E00F9039
:101D20000F900F900F900F90CF91DF911F910F9117
:101D3000FF90EF90DF90CF90BF90AF909F908F90EB
:101D40007F906F905F904F900895BF92CF92DF92F7
:101D5000EF92FF920F931F936C01FC01B080E18022
:101D60000E946E4620E831E541E050E00E946A574B
:101D70008B2D8F77280F311D411D511DFF2400E051
:101D800010E0CA01B901A80197010E946A57F0E862
:101D9000BF22B62AF601B0821F910F91FF90EF90FB
:101DA000DF90CF90BF9008956F927F928F929F9215
:101DB000AF92BF92CF92DF92EF92FF920F931F9359
:101DC0004C01FC01708061800E946E46A62CBB24F1
:101DD000CC24DD24BFE7EB2EE720FF24E60CF11C2A
:101DE0000027F7FC0095102F20E831E541E050E096
:101DF0000E946A57CA01B901A60195010E946A575B
:101E0000E61AF70A080B190BC801B701A6019501DC
:101E10000E946A57F0E87F22762AF40170821F91AF
:101E20000F91FF90EF90DF90CF90BF90AF909F9079
:101E30008F907F906F900895EF92FF921F93CF93B2
:101E4000DF93182F7B010E946E469B01AC01C12FCE
:101E5000D0E02F5F3F4F4F4F5F4FCE01880F991F4C
:101E6000880F991FFC01E85DF84F2083318342837E
:101E70005383FC01E851F84FE114F10449F48EEF6B
:101E80009FEFAFEFBFEF80839183A283B3830DC039
:101E9000C701AA2797FDA095BA2F280F391F4A1FFF
:101EA0005B1F2083318342835383C855D74F83E61A
:101EB00088838091FB0888608093FB08DF91CF9135
:101EC0001F91FF90EF9008958F929F92AF92BF92D3
:101ED000CF92DF92EF92FF920F931F93CF93DF93F6
:101EE0008C010E5F1F4F20E030E006C0F901EF517A
:101EF000F94F90830F5F1F4FE22FD8019C91892FDC
:101F000080538A3028F42F5F3F4F2530310571F719
:101F1000F0E0EE51F94F108282EE96E00E94ED075C
:101F2000EC0197FD00C18091FE0890E08C179D07A1
:101F30000CF4F9C0F80180818D3309F057C0209767
:101F400009F4F1C08091FB0884FFEDC02197C8011E
:101F500001962181203379F40E946E46EC2FF0E047
:101F6000EE0FFF1FEE0FFF1FE851F84F60837183E4
:101F70008283938319C0213309F0D5C062EE76E0E5
:101F800040E320E031E00E940D41882319F460E035
:101F900070E007C082EE96E00E94ED07BC0197FD5D
:101FA000C2C08C2F0E941C0F00D000D000D0EDB713
:101FB000FEB7319683E197E0ADB7BEB712969C931A
:101FC0008E93119789ED91E09383828380E790E06F
:101FD000958384830E94093B81E0EDB7FEB7369676
:101FE0000FB6F894FEBF0FBEEDBF9EC000D000D06C
:101FF00000D0EDB7FEB7319683E197E0ADB7BEB73D
:1020000012969C938E93119786ED91E09383828331
:1020100080E790E0958384830E94093BEDB7FEB78B
:1020200036960FB6F894FEBF0FBEEDBF209721F491
:102030008091FE0890E003C08C2F9C2F9150C0E04F
:10204000D0E0E92EFF24082F10E073E1C72E77E0DF
:10205000D72E60ED862E61E0962E53EDA52E51E031
:10206000B52E58C09091FB0890FF39C091FD37C044
:1020700080916002882311F092FD31C000D000D021
:1020800000D0ADB7BEB71196EDB7FEB7D282C18210
:102090001396BC92AE921297F90143E0F595E7953D
:1020A0004A95E1F7E150F74F808190E0277030705A
:1020B00002C0959587952A95E2F7817090701596E4
:1020C0009C938E9314970E94093B2DB73EB72A5FCD
:1020D0003F4F0FB6F8943EBF0FBE2DBF1AC000D0C1
:1020E00000D000D0EDB7FEB73196ADB7BEB71296AF
:1020F000DC92CE92119793828282158214820E9482
:10210000093BEDB7FEB736960FB6F894FEBF0FBE8B
:10211000EDBF21969E012E0D3F1D201731070CF4B7
:10212000A1CF81E001C080E0DF91CF911F910F919D
:10213000FF90EF90DF90CF90BF90AF909F908F90E7
:102140000895BF92CF92DF92EF92FF920F931F9369
:10215000CF93DF9300D000D003E117E0ADB7BEB757
:1021600012961C930E9311978BE19AE014969C9310
:102170008E9313970E94093BFF240F900F900F90AE
:102180000F90B02EE12EB2EECB2EB6E0DB2E05E1A5
:102190001AE021C08F2D62EE76E00E94422800D026
:1021A00000D000D0EDB7FEB73196ADB7BEB71196EF
:1021B000BC9211971296EC9213830283D582C4824B
:1021C0000E94093BF394EDB7FEB736960FB6F8942C
:1021D000FEBF0FBEEDBF8091FE08C3E1D7E0F81649
:1021E000C8F200D000D0ADB7BEB71296DC93CE9344
:1021F000119780E19AE014969C938E9313970E9416
:10220000093B0F900F900F900F908E819F812C8132
:102210003D81821B930B60E140E00E94ED35DF9130
:10222000CF911F910F91FF90EF90DF90CF90BF90D3
:1022300008954F925F926F927F928F929F92AF928A
:10224000BF92CF92DF92EF92FF920F931F93DF9393
:10225000CF930F92CDB7DEB70E946E465B016C0143
:102260002DB73EB7285030400FB6F8943EBF0FBE92
:102270002DBFEDB7FEB7319603E117E0ADB7BEB79E
:1022800012961C930E93119782EE94E093838283AF
:1022900080E790E09583848387EF90E0978386833F
:1022A0000E94093BEDB7FEB738960FB6F894FEBF13
:1022B0000FBEEDBF0E94A1101092160710921507D5
:1022C00084E993E0909318078093170790931A0777
:1022D000809319072DB73EB72A5030400FB6F894B7
:1022E0003EBF0FBE2DBFEDB7FEB73196ADB7BEB73F
:1022F00012961C930E9311978DEC94E09383828336
:102300008BEC90E095838483A682B782C086D186C9
:102310000E94093B0F900F90EDB7FEB73196ADB715
:10232000BEB712961C930E93119783EB94E09383A0
:1023300082838091FD08848315828091D4018683F5
:1023400017820E94093B90E0EDB7FEB738960FB6B2
:10235000F894FEBF0FBEEDBF78010FEA14E023C072
:1023600000D000D000D0EDB7FEB73196ADB7BEB704
:102370001196EC9211971296FC9213830283A92F67
:10238000B0E0A150B74F8C918483158299830E944D
:10239000093B99819F5FEDB7FEB736960FB6F8946B
:1023A000FEBF0FBEEDBF8091FD0823E1622E27E046
:1023B000722E9817A8F200D000D0ADB7BEB7129613
:1023C0007C926E92119783EA94E014969C938E937C
:1023D00013970E94093B99240F900F900F900F9034
:1023E000C301762C892E8AE9482E84E0582E66C0D7
:1023F000A92DB0E0FD01E855F74F60816623A9F1F2
:10240000CD01880F991F880F991FFC01E85DF84FD7
:10241000E080F18002811381FC01E851F84FAE1495
:10242000BF04C006D10648F020813181428153812A
:102430002A193B094C095D0908C02081318142817C
:1024400053812E193F09400B510BAA0FBB1FAA0F36
:10245000BB1FA851B84F8D919D910D90BC91A02D9F
:102460008E5F9F4FAF4FBF4F21F420E030E040E040
:1024700050E08DB79EB70A970FB6F8949EBF0FBE77
:102480008DBFEDB7FEB73196ADB7BEB711967C9252
:10249000119712968C92538242826483158226830E
:1024A0003783408751870E94093B9394EDB7FEB76D
:1024B0003A960FB6F894FEBF0FBEEDBF8091FE08AE
:1024C000981608F495CF2DB73EB72A5130400FB675
:1024D000F8943EBF0FBE2DBFEDB7FEB7319603E1B6
:1024E00017E0ADB7BEB712961C930E93119788E410
:1024F00094E0938382838091FB08817084831582AA
:102500008091FB0886958170868317828091FB08F5
:10251000869586958170808711868091FB088295CB
:1025200081708287138680910B0990910C09A0918C
:102530000D09B0910E0984879587A687B78780918A
:102540004B02808B118A80916002828B138A80916A
:102550006E02848B158A80917C02868B178A80E6B6
:1025600090E0918F808F0E94093BEDB7FEB73C96BB
:102570000FB6F894FEBF0FBEEDBF3196ADB7BEB734
:1025800012961C930E93119786E294E093838283B4
:10259000809120078483158280912107868317828A
:1025A000809122079091230791878087809124074B
:1025B00090912507A0912607B091270782879387DE
:1025C000A487B5870E94093BEDB7FEB738960FB6D2
:1025D000F894FEBF0FBEEDBF3196ADB7BEB71296F1
:1025E0001C930E93119782E094E09383828380E89A
:1025F00090E0958384830E94093BEDB7FEB7369641
:102600000FB6F894FEBF0FBEEDBF81E00F90CF91E3
:10261000DF911F910F91FF90EF90DF90CF90BF90CF
:10262000AF909F908F907F906F905F904F900895A4
:10263000FF920F931F93CF93DF938C010E9472360A
:10264000109216071092150784E993E090931807EB
:102650008093170790931A0780931907A8014B5F7F
:102660005F4FD80115968C91803221F4CA010E94E7
:1026700019116EC0C1E8D1E0A0E0B0E0682F772763
:1026800067FD7095FA2EE881F981849190E08617B4
:10269000970709F06CC03196249130E0FA018181EE
:1026A000992787FD90952817390709F060C0AA0F70
:1026B000BB1FAA0FBB1FAD57BE4FED91FC91CA01C6
:1026C0000995882301F500D000D000D0EDB7FEB702
:1026D000319683E197E0ADB7BEB712969C938E9387
:1026E00011978DEC91E09383828382E291E0958350
:1026F00084830E94093BEDB7FEB736960FB6F89477
:10270000FEBF0FBEEDBFF3E1FF1611F58091FB0890
:1027100086FF1EC0402FE2EEF6E0C801DC0101C0DA
:1027200081939A2F941B15968C911597803229F0DE
:10273000119627E0E230F20799F7E92FF0E0EE5129
:10274000F94F108282EE96E061E00E94640A17C0A1
:102750008091190790911A07209117073091180757
:10276000821B930B61E140E00E94ED3508C0F394B9
:1027700011962496A331B10509F084CFC4CFDF911F
:10278000CF911F910F91FF900895BF92CF92DF924A
:10279000EF92FF920F931F93CF93DF932DB73EB726
:1027A000285030400FB6F8943EBF0FBE2DBFEDB796
:1027B000FEB7319603E117E0ADB7BEB712961C9392
:1027C0000E93119782EB97E09383828380E790E0EA
:1027D0009583848387EF90E0978386830E94093BEB
:1027E000EDB7FEB738960FB6F894FEBF0FBEEDBF3B
:1027F0000E94A110109216071092150784E993E029
:10280000909318078093170790931A0780931907DE
:102810002DB73EB72A5030400FB6F8943EBF0FBEDA
:102820002DBFEDB7FEB73196ADB7BEB712961C936C
:102830000E9311978EE897E0938382838091FD0831
:102840008483158280914B028683178280917C025B
:10285000808711860E94093BDD24E12C44E0F42EA0
:10286000EDB7FEB73A960FB6F894FEBF0FBEEDBFB8
:10287000B02EC12E0AE817E033C0F999FECFF2BCA2
:10288000E1BCF89A90B5F999FECF0894E11CF11CCF
:10289000F2BCE1BCF89A80B5D92FC0E000D000D0DE
:1028A00000D0EDB7FEB73196ADB7BEB71196BC926A
:1028B00011971296CC92138302839E01280F311D2B
:1028C000358324830E94093BD3940894E11CF11CB6
:1028D0008DB79EB706960FB6F8949EBF0FBE8DBFFC
:1028E0008091FE08D81608F4C8CF00D000D003E1CC
:1028F00017E0ADB7BEB712961C930E9311978CE7F5
:1029000097E014969C938E9313970E94093B00D0F6
:10291000EDB7FEB73196ADB7BEB712961C930E93C6
:10292000119786E597E09383828380E890E0958312
:1029300084830E94093BEDB7FEB736960FB6F89434
:10294000FEBF0FBEEDBF81E0DF91CF911F910F91D0
:10295000FF90EF90DF90CF90BF900895CF92DF92DD
:10296000FF920F931F93DF93CF930F92CDB7DEB7F4
:1029700000D000D000D0EDB7FEB7319603E117E0EC
:10298000ADB7BEB712961C930E93119784E99AE0E7
:102990009383828380E790E0958384830E94093B40
:1029A000EDB7FEB736960FB6F894FEBF0FBEEDBF7B
:1029B0000E94A110109216071092150784E993E067
:1029C000909318078093170790931A07809319071D
:1029D0002DB73EB72C5030400FB6F8943EBF0FBE17
:1029E0002DBFEDB7FEB73196ADB7BEB712961C93AB
:1029F0000E9311978BE69AE0938382838091FD0872
:102A00008483158280E190E09783868380914B02D6
:102A10008087118680917C02828713860E94093B01
:102A2000EDB7FEB738960FB6F894FEBF0FBEEDBFF8
:102A3000128301838FE59AE0948383830E94093B8C
:102A400090E00F900F900F900F90F02E012F5BE50C
:102A5000C52E5AE0D52E23C000D000D000D0EDB74F
:102A6000FEB73196ADB7BEB71196FC92119712968C
:102A70000C93D382C282A92FB0E0AB5FB64F8C918A
:102A80008483158299830E94093B99819F5FEDB7EA
:102A9000FEB736960FB6F894FEBF0FBEEDBF80911D
:102AA000FD089817C8F200D000D000D0EDB7FEB7EF
:102AB000319683E197E0ADB7BEB712969C938E93A3
:102AC000119788E29AE09383828380E890E095836F
:102AD00084830E94093BEDB7FEB736960FB6F89493
:102AE000FEBF0FBEEDBF81E00F90CF91DF911F9130
:102AF0000F91FF90DF90CF900895BF92CF92DF9219
:102B0000EF92FF920F931F93CF93DF9300D000D0EB
:102B100000D0EDB7FEB7319603E117E0ADB7BEB711
:102B200012961C930E93119788ED9AE093838283FB
:102B30008FEA90E0958384830E94093B0F900F9069
:102B4000EDB7FEB7128301838CEC9AE09483838304
:102B50000E94093BFF240F900F900F900F90B02E12
:102B6000E12E72EEC72E76E0D72E06EC1AE021C0D9
:102B70008F2D62EE76E00E94422800D000D000D077
:102B8000EDB7FEB73196ADB7BEB71196BC921197AF
:102B90001296EC9213830283D582C4820E94093B71
:102BA000F394EDB7FEB736960FB6F894FEBF0FBE9E
:102BB000EDBF8091FE08C3E1D7E0F816C8F200D05F
:102BC00000D0ADB7BEB71296DC93CE93119783EBCE
:102BD0009AE014969C938E9313970E94093B00E011
:102BE0000F900F900F900F90CE01DC2E192F6FEAEF
:102BF000E62E6AE0F62E21C000D000D000D0EDB75E
:102C0000FEB73196ADB7BEB71196DC92119712960A
:102C10001C93F382E282A02FB0E0AB5FB64F8C91A1
:102C2000848315820E94093B0F5FEDB7FEB736968D
:102C30000FB6F894FEBF0FBEEDBF8091FD08C3E153
:102C4000D7E00817C8F200D000D000D0EDB7FEB72B
:102C50003196ADB7BEB71296DC93CE9311978FE93C
:102C60009AE09383828380E190E0958384830E943D
:102C7000093BEDB7FEB736960FB6F894FEBF0FBE10
:102C8000EDBF81E0DF91CF911F910F91FF90EF9009
:102C9000DF90CF90BF9008959C0180917C028823A3
:102CA00011F081E00895C90162EE76E040E322E090
:102CB00031E00E940D41882331F082EE96E00E94BF
:102CC0004129811181E008954F925F926F927F9226
:102CD0008F929F92AF92BF92CF92DF92EF92FF922C
:102CE0000F931F93DF93CF93CDB7DEB7E5970FB662
:102CF000F894DEBF0FBECDBFF3E0AF2EB12CA80E0F
:102D0000B91EC5010E944C16882309F436C15090A3
:102D1000D4014090DB010DEC11E0EE24CC24DD2445
:102D20004E010894811C911CE2E06E2E712C6C0EF9
:102D30007D1E2C2D9D2DD80116968C91169781FF06
:102D40003BC011968C911197813009F41C92D401EB
:102D5000ECEFF2E085E001900D928150E1F7822FD7
:102D6000B3014AE050E00E94F108C50162EE76E04E
:102D700040E394010E940D418823F1F0F801F180B5
:102D8000F1E0FF1619F4D801FC9216C082EE96E02D
:102D90000E94ED079C01B4E1CB1611F4245C3F4F77
:102DA00037FD08C08F2D90E0821793071CF0F801C3
:102DB000208302C0EE24E3940894C11CD11C095F57
:102DC0001F4FF2E2CF16D10409F0B3CFC50162EE76
:102DD00076E040E325E031E00E940D41882351F088
:102DE00082EE96E00E94594180E690E062EE76E045
:102DF0000E941C29C50162EE76E040E329E031E043
:102E00000E940D418823C1F082EE96E00E94594154
:102E100082EE96E00E940B08162F072FF82ED92E6F
:102E20000E9441468091FB0885FF06C0612F702FEC
:102E30008F2D9D2D0E944F34EE2089F000D000D0C0
:102E400000D0EDB7FEB7319683E197E0ADB7BEB7DE
:102E500012969C938E9311978CEA92E0B5C00E94D3
:102E6000F828C50162EE76E040E32DE031E00E94F3
:102E70000D41882309F444C08E010A5F1F4FC5012C
:102E8000B80140E321E131E00E940D41882309F4BB
:102E90008BC082EE96E0B80140E150E00E945F08EE
:102EA000009709F081C080E490E062EE76E00E9435
:102EB0001C292DB73EB7285030400FB6F8943EBFBE
:102EC0000FBE2DBFEDB7FEB7319683E197E0ADB7EA
:102ED000BEB712969C938E93119784E892E09383E9
:102EE000828380E790E09583848382E791E09783F3
:102EF00086830E94093B81E0EDB7FEB7389670C02B
:102F00002DB73EB7285030400FB6F8943EBF0FBEE5
:102F10002DBFEDB7FEB7319683E197E0ADB7BEB7F1
:102F200012969C938E9311978AE092E0938382830A
:102F300080E790E09583848382E791E0978386839E
:102F40000E94093BEDB7FEB738960FB6F894FEBF66
:102F50000FBEEDBF8091D401851531F4442061F49A
:102F60008091DB01882341F010921B0710921C070F
:102F700010921D0710921E0781E0E5960FB6F89497
:102F8000DEBF0FBECDBFCF91DF911F910F91FF909C
:102F9000EF90DF90CF90BF90AF909F908F907F90F9
:102FA0006F905F904F90089500D000D000D0EDB7A3
:102FB000FEB7319683E197E0ADB7BEB712969C930A
:102FC0008E93119786E392E09383828380E790E06B
:102FD000958384830E94093B81E0EDB7FEB7369666
:102FE0000FB6F894FEBF0FBEEDBFC7CF0F931F9370
:102FF000DF93CF93CDB7DEB7C058D0400FB6F8946B
:10300000DEBF0FBECDBF8C010D5F1F4FC8010E94F8
:103010004C16882309F440C0C8018E010F5F1F4F72
:10302000B80140E825E131E00E940D41882341F0DC
:10303000C8010E94594180E890E0B8010E941C2913
:103040002DB73EB7285030400FB6F8943EBF0FBEA4
:103050002DBFEDB7FEB7319683E197E0ADB7BEB7B0
:1030600012969C938E93119785EF92E093838283BF
:1030700080E790E09583848382E791E0978386835D
:103080000E94093B81E02DB73EB7285F3F4F0FB646
:10309000F8943EBF0FBE2DBFC058DF4F0FB6F89457
:1030A000DEBF0FBECDBFCF91DF911F910F9108956D
:1030B0008F929F92AF92BF92CF92DF92FF920F9327
:1030C0001F93DF93CF9300D000D0CDB7DEB713E0CE
:1030D000C12ED12CC80ED91EC6010E944C168823C1
:1030E00009F483C083E789831A821B821C8210E063
:1030F000B2E08B2E912C8C0E9D1E5E010894A11CBB
:10310000B11C1AC0812F90E0B4014AE050E00E9447
:10311000F108C60162EE76E040E395010E940D41A0
:10312000882349F082EE96E00E945941812F62EE99
:1031300076E00E9467281F5F8091FE08181710F341
:103140008DE68983FF24A2E08A2E912C8C0E9D1E91
:103150005E010894A11CB11C1AC00F2D10E0C8011B
:10316000B4014AE050E00E94F108C60162EE76E048
:1031700040E395010E940D41882341F082EE96E0E4
:103180000E94ED070B5F164FD8018C93F39480914A
:10319000FD08F81610F30E949128EDB7FEB7389796
:1031A0000FB6F894FEBF0FBEEDBF319683E197E0F6
:1031B000ADB7BEB712969C938E9311978BEE99E0A4
:1031C0009383828380E790E09583848382E791E014
:1031D000978386830E94093B81E0EDB7FEB738965E
:1031E0000FB6F894FEBF0FBEEDBF0F900F900F907B
:1031F0000F90CF91DF911F910F91FF90DF90CF90B3
:10320000BF90AF909F908F9008958F929F92AF92B2
:10321000BF92CF92DF92EF92FF920F931F93CF93C3
:10322000DF93EC017A018B01CB01BA010E945B456F
:103230004C01C801B7010E9455455C01888988236B
:1032400009F481C0D880D7FE21C0C98021E02C15A7
:10325000E8F4C801B70120E831E541E050E00E9400
:103260006A57CA01B9012C2D30E040E050E00E94BD
:103270006A572FE7D2222D2D30E040E050E0621750
:1032800073078407950709F05EC031C0C801B70114
:103290000E944945288130E090E0059667E070E0A3
:1032A0000E94575702C0359527958A95E2F720FF6F
:1032B0004AC0C801B7010E944F45D82E888187FFB8
:1032C00016C08981882319F4D0FE11C03CC081301A
:1032D00071F48FE1D816B9F12DE1D21609F042C090
:1032E000C801B7010E9443450297E1F52CC08CE369
:1032F00090E0889E9001899E300D989E300D11249B
:103300002A0D3B1D4A815B8124173507E0F08C8133
:103310009D8182179307B8F0EE81FF81309799F075
:10332000241B350B40E0C901BF010E9443576E9F2B
:10333000C0016F9F900D7E9F900D112482179307FF
:1033400019F441E001C040E0842FDF91CF911F913B
:103350000F91FF90EF90DF90CF90BF90AF909F9034
:103360008F900895D0FCC3CFEECF982F9B01809112
:103370001F07981768F461E1969FB00111246859FE
:103380007B4FC90141E150E024E639E00E946D081D
:103390000895CF92DF92EF92FF920F931F93DF93E6
:1033A000CF93CDB7DEB762970FB6F894DEBF0FBEEE
:1033B000CDBF8C010D5F1F4FC8010E945941C8014C
:1033C00062EE76E040E329E131E00E940D4188237E
:1033D00009F42BC182EE96E00E94ED077C012FEFED
:1033E0008F3F92070CF421C180911F0790E0E816EF
:1033F000F9060CF01AC18DB79EB708970FB6F8946E
:103400009EBF0FBE8DBFEDB7FEB7319603E117E04B
:10341000ADB7BEB712961C930E93119787E097E055
:103420009383828380E790E09583848387EF90E0A5
:10343000978386830E94093BEDB7FEB738960FB697
:10344000F894FEBF0FBEEDBF0E94A11010921607A8
:103450001092150784E993E090931807809317075B
:1034600090931A07809319072DB73EB72A50304022
:103470000FB6F8943EBF0FBE2DBFEDB7FEB7319625
:10348000ADB7BEB712961C930E93119788EE96E0D7
:10349000938382838091FD0884831582F782E6827C
:1034A00080917C02808711860E94093BEDB7FEB7B0
:1034B0003A960FB6F894FEBF0FBEEDBFFFEFEF16C2
:1034C000FFEFFF0609F48FC08E2D7E010894E11CEA
:1034D000F11CB7010E94B5198A81823018F0C7012A
:1034E0000E94D40E2DB73EB7225130400FB6F8944B
:1034F0003EBF0FBE2DBFEDB7FEB7319603E117E01B
:10350000ADB7BEB712961C930E93119789EC96E057
:103510009383828389898483158289818683178234
:103520008A81808711868B819C81938782878D8198
:103530009E81958784878F819885978786878985DF
:103540009A85918B808B0E94093B90E0EDB7FEB786
:1035500072960FB6F894FEBF0FBEEDBF680105EC82
:10356000E02E06E0F02E8E01055F1F4F22C000D036
:1035700000D000D0EDB7FEB73196ADB7BEB711960B
:10358000CC9211971296DC92F382E282D801A90FB5
:10359000B11D8C91848315829A8B0E94093B9A8974
:1035A0009F5FEDB7FEB736960FB6F894FEBF0FBE1D
:1035B000EDBF8091FD089817D0F200D000D083E1D4
:1035C00097E0ADB7BEB712969C938E93119782EC9D
:1035D00096E014969C938E9313970E94093B0F904C
:1035E0000F900F900F9000D000D000D0EDB7FEB735
:1035F000319683E197E0ADB7BEB712969C938E9358
:10360000119781E996E09383828380E890E0958327
:1036100084830E94093B81E0EDB7FEB736960FB672
:10362000F894FEBF0FBEEDBF01C080E062960FB6FA
:10363000F894DEBF0FBECDBFCF91DF911F910F91E8
:10364000FF90EF90DF90CF9008952F923F924F928E
:103650005F926F927F928F929F92AF92BF92CF9222
:10366000DF92EF92FF920F931F93DF93CF93CDB72B
:10367000DEB761970FB6F894DEBF0FBECDBF00D0A6
:1036800000D000D0EDB7FEB7319603E117E0ADB73B
:10369000BEB712961C930E9311978AE198E093831C
:1036A00082838FEA90E0958384830E94093B00D057
:1036B00000D0EDB7FEB73196ADB7BEB712961C93EA
:1036C0000E93119780EF97E09383828380911F0779
:1036D000848315828091FD088683178286E390E0BB
:1036E000918780870E94093BDD24EDB7FEB73A96AB
:1036F0000FB6F894FEBF0FBEEDBF4E010894811CBB
:10370000911CC02E012F2BE0222E312C2C0E3D1EA1
:103710004C2C512E93ED692E97E0792E84E9A82E3A
:1037200083E0B82E9AC08D2DB4010E94B5198A810C
:10373000823018F0C4010E94D40EED2CFF248DB706
:103740009EB744970FB6F8949EBF0FBE8DBFEDB7DE
:10375000FEB73196ADB7BEB71196CC9211971296BF
:103760000C938AED97E093838283F582E4828989C2
:10377000868317828981808711868A818287138652
:103780008B819C81958784878D819E819787868791
:103790008F819885918B808B89859A85938B828B7D
:1037A0000E94093B10E0ADB7BEB754961DC000D0D3
:1037B00000D000D0EDB7FEB73196ADB7BEB71196C9
:1037C000CC92119712960C9386ED97E093838283A7
:1037D000D101A10FB11D8C91848315820E94093BF8
:1037E0001F5FADB7BEB716960FB6F894BEBF0FBE3B
:1037F000ADBF8091FD081817D0F200D000D0EDB712
:10380000FEB741825282748263820E94093BF3E0D8
:10381000EF22FF240F900F900F900F9083E0E81697
:10382000F104D1F48091190790911A07209117079C
:1038300030911807821B930B60E140E00E94ED3548
:103840001092160710921507B0921807A09217074A
:10385000B0921A07A0921907D39480911F07D81627
:1038600008F461CF00D000D083E197E0ADB7BEB7D8
:1038700012969C938E9311978FEB97E014969C93DE
:103880008E9313970E94093B0F900F900F900F900B
:1038900081E061960FB6F894DEBF0FBECDBFCF9129
:1038A000DF911F910F91FF90EF90DF90CF90BF902D
:1038B000AF909F908F907F906F905F904F903F90D0
:1038C0002F9008952F923F924F925F926F927F9226
:1038D0008F929F92AF92BF92CF92DF92EF92FF9220
:1038E0000F931F93DF93CF93CDB7DEB761970FB6DA
:1038F000F894DEBF0FBECDBF8DB79EB70C970FB645
:10390000F8949EBF0FBE8DBFEDB7FEB7319603E1B1
:1039100017E0ADB7BEB712961C930E9311978CEBC0
:1039200099E09383828380911F078483158280911D
:10393000FD088683178280917C028087118686E34A
:1039400090E0938782870E94093BDD24EDB7FEB7A4
:103950003C960FB6F894FEBF0FBEEDBF4E01089423
:10396000811C911CC02E012F5BE0252E312C2C0ECA
:103970003D1E4C2C512E48E9642E49E0742E34E94A
:10398000A32E33E0B32E9AC08D2DB4010E94B51939
:103990008A81823018F0C4010E94D40EED2CFF24DD
:1039A0008DB79EB744970FB6F8949EBF0FBE8DBFDC
:1039B000EDB7FEB73196ADB7BEB71196CC92119761
:1039C00012960C938FE999E093838283F582E482C7
:1039D0008989868317828981808711868A81828777
:1039E00013868B819C81958784878D819E819787A3
:1039F00086878F819885918B808B89859A85938B1B
:103A0000828B0E94093B10E0ADB7BEB754961DC033
:103A100000D000D000D0EDB7FEB73196ADB7BEB73D
:103A20001196CC92119712960C938BE999E093839F
:103A30008283D101A10FB11D8C91848315820E94D4
:103A4000093B1F5FADB7BEB716960FB6F894BEBF61
:103A50000FBEADBF8091FD081817D0F200D000D086
:103A6000EDB7FEB741825282748263820E94093BA5
:103A7000F3E0EF22FF240F900F900F900F9083E060
:103A8000E816F104D1F48091190790911A0720915A
:103A9000170730911807821B930B60E140E00E94EA
:103AA000ED351092160710921507B0921807A092E4
:103AB0001707B0921A07A0921907D39480911F0795
:103AC000D81608F461CF00D000D083E197E0ADB7FD
:103AD000BEB712969C938E9311978DE899E0149639
:103AE0009C938E9313970E94093B0F900F900F9019
:103AF0000F9061960FB6F894DEBF0FBECDBFCF9189
:103B0000DF911F910F91FF90EF90DF90CF90BF90CA
:103B1000AF909F908F907F906F905F904F903F906D
:103B20002F9008952F923F924F925F926F927F92C3
:103B30008F929F92AF92BF92CF92DF92EF92FF92BD
:103B40000F931F93DF93CF9300D0CDB7DEB78C01D7
:103B50000D5F1F4FC8010E9459410E946E465B01D4
:103B60006C010E943A452C01C601B5010E944345F3
:103B70003C01C601B5010E944F454C01C601B5018B
:103B80000E945B459A838983C601B5010E94554511
:103B90001C01C80162EE76E040E32DE131E00E94B5
:103BA0000D41882361F082EE96E00E94ED074C0102
:103BB000009729F4C601B5010E944F454C01C80188
:103BC00062EE76E040E32FE131E00E940D41882370
:103BD00029F082EE96E00E94ED073C01C80162EEFA
:103BE00076E040E321E231E00E940D41882329F094
:103BF00082EE96E00E94ED072C0100D000D000D0AC
:103C0000EDB7FEB73196A3E1EA2EA7E0FA2EADB7E5
:103C1000BEB71296FC92EE9211978BE596E09383D5
:103C2000828380E790E0958384830E94093BEDB70F
:103C3000FEB736960FB6F894FEBF0FBEEDBF0E94DA
:103C4000A110109216071092150784E993E0909343
:103C500018078093170790931A07809319072DB7B9
:103C60003EB72A5130400FB6F8943EBF0FBE2DBF6D
:103C70000DB71EB70F5F1F4FADB7BEB71296FC92C0
:103C8000EE92119784E096E0F8019383828380910D
:103C90003D028483158280914B0286831782809136
:103CA0006E028087118680914402828713868091FC
:103CB0005202848715868091590286871786C6012D
:103CC000B50120E831E541E050E00E946A57D80193
:103CD00051963C932E9350978CE390E0E981FA81C2
:103CE0009C01E29FC001E39F900DF29F900D112473
:103CF000820D931D53969C938E93529755969C924A
:103D00008E92549757967C926E92569759965C92E3
:103D10004E9258970E94093B4DB75EB74A5E5F4F7F
:103D20000FB6F8945EBF0FBE4DBFADB7BEB71296CB
:103D3000FC92EE92119788EF95E014969C938E93E7
:103D400013970E94093B00E00F900F900F900F9087
:103D5000BE2CEF2C74EFC72E75E0D72E21C000D0FB
:103D600000D000D0EDB7FEB73196ADB7BEB7119613
:103D7000BC9211971296EC92D382C282A02FB0E02F
:103D8000AB5FB64F8C91848315820E94093B0F5F15
:103D9000EDB7FEB736960FB6F894FEBF0FBEEDBF77
:103DA0008091FD0863E1862E67E0962E0817B8F231
:103DB00000D000D0ADB7BEB712969C928E921197EC
:103DC00080EF95E014969C938E9313970E94093B85
:103DD0000F900F900F900F900E94621C00D000D0A7
:103DE00000D0EDB7FEB73196ADB7BEB712969C9234
:103DF0008E92119788EC95E09383828380E890E01F
:103E0000958384830E94093BEDB7FEB736960FB6C3
:103E1000F894FEBF0FBEEDBF81E00F900F90CF91E1
:103E2000DF911F910F91FF90EF90DF90CF90BF90A7
:103E3000AF909F908F907F906F905F904F903F904A
:103E40002F9008950F931F938DB79EB708970FB6C5
:103E5000F8949EBF0FBE8DBFEDB7FEB7319603E15C
:103E600017E0ADB7BEB712961C930E9311978CE373
:103E700097E09383828380E790E09583848387EF44
:103E800090E0978386830E94093B8DB79EB7089682
:103E90000FB6F8949EBF0FBE8DBF0E94A110109266
:103EA00016071092150784E993E090931807809302
:103EB000170790931A07809319070E94621C00D07D
:103EC00000D000D0EDB7FEB73196ADB7BEB71296B1
:103ED0001C930E93119784E197E09383828380E88B
:103EE00090E0958384830E94093B8DB79EB7069628
:103EF0000FB6F8949EBF0FBE8DBF81E01F910F914A
:103F00000895DF92EF92FF920F931F93DF93CF9369
:103F1000CDB7DEB761970FB6F894DEBF0FBECDBF49
:103F200020911F07821708F043C0222309F440C0E4
:103F300090E001968C0124E0000F111F2A95E1F713
:103F4000080F191F08591B4FB1E1DB2E7E010894A1
:103F5000E11CF11C13C0C701B80141E150E024E6A7
:103F600039E00E946D08C8014197B70141E150E076
:103F70002CE639E00E94AF080F5E1F4F20911F070B
:103F80002D9DC001112488599B4F0817190718F35C
:103F9000215020931F07F999FECF1FBA86E694E0BF
:103FA00092BD81BD20BD0FB6F894FA9AF99A0FBE62
:103FB00061960FB6F894DEBF0FBECDBFCF91DF91F3
:103FC0001F910F91FF90EF90DF900895CF93DF93B3
:103FD000EC012396CE010E945941CE010E944C165D
:103FE000882309F450C0CE0162EE76E040E329E177
:103FF00031E00E940D41882309F445C082EE96E02D
:104000000E94ED079C018FEF2F3F380781F410923B
:104010001F07F999FECF1FBA86E694E092BD81BDD5
:1040200010BC0FB6F894FA9AF99A0FBE09C08091A5
:104030001F0790E02817390734F5822F0E94811F4F
:1040400000D000D000D0EDB7FEB7319683E197E005
:10405000ADB7BEB712969C938E93119786E696E005
:104060009383828380E790E0958384830E94093B59
:1040700081E02DB73EB72A5F3F4F0FB6F8943EBFA1
:104080000FBE2DBF01C080E0DF91CF910895982F22
:1040900080911F07981760F481E1989FC001112457
:1040A00088599B4F41E150E02CE639E00E94AF086F
:1040B0000895BC0190911F079633F0F481E1989F19
:1040C000C001112488599B4F41E150E02CE639E0B2
:1040D0000E94AF0820911F072F5F20931F07F999B7
:1040E000FECF1FBA86E694E092BD81BD20BD0FB61B
:1040F000F894FA9AF99A0FBE0895BF92CF92DF9280
:10410000EF92FF920F931F93DF93CF93CDB7DEB75C
:1041100063970FB6F894DEBF0FBECDBF7C018C0154
:104120000D5F1F4FC8010E945941C8010E944C16E3
:10413000882309F403C1C80162EE76E040E329E177
:1041400031E00E940D41882309F4F8C082EE96E028
:104150000E94ED076C012FEF8F3F92070CF4EEC029
:1041600080911F0790E0C816D9060CF0E7C01A83AB
:10417000098387E690E0E80EF91E0DC0C80163E2EE
:1041800071E043E050E00E945F08009779F00F5F14
:104190001F4F1A83098309811A81D8018C918823C2
:1041A00009F4CCC00E151F0548F3C8C00D5F1F4FA2
:1041B0001A8309838E010F5F1F4FC8010E942F0CC5
:1041C0008B8BC8010E942F0C8B83C8010E942F0C7F
:1041D0008C83C8010E942F0C9E838D83C8010E948E
:1041E0002F0C98878F83C8010E942F0C9A8789878C
:1041F000C8010E942F0C9C878B87FF24B02EE12ED4
:104200008E01035F1F4F09C08B2D9E2D0E942F0C26
:10421000F801EF0DF11D8083F3948091FD08F816ED
:1042200098F306C0FC01EF0DF11D1082F39402C05B
:10423000CE010D96B5E0BF15A8F78C81823020F035
:10424000CE0103960E94A50E00D000D000D0EDB79D
:10425000FEB7319603E117E0ADB7BEB712961C93D7
:104260000E9311978DEB95E09383828380E790E026
:10427000958384830E94093BEDB7FEB736960FB64F
:10428000F894FEBF0FBEEDBFBE016D5F7F4FFFEF25
:10429000CF16FFEFDF06C1F4CB010E94592000D0FA
:1042A00000D0ADB7BEB712961C930E93119780EA5B
:1042B00095E014969C938E9313970E94093B0F9060
:1042C0000F900F900F9022C08C2D0E94472000D09D
:1042D00000D000D0EDB7FEB73196ADB7BEB712969D
:1042E0001C930E93119782E895E093838283089440
:1042F000C11CD11CD582C4820E94093BEDB7FEB718
:1043000036960FB6F894FEBF0FBEEDBF00D000D0BA
:1043100083E197E0ADB7BEB712969C938E93119749
:1043200081E695E014969C938E9313970E94093B27
:1043300081E00F900F900F900F9001C080E0639686
:104340000FB6F894DEBF0FBECDBFCF91DF911F91A6
:104350000F91FF90EF90DF90CF90BF9008950E9453
:10436000CC280E94432DA8EAB8E080E090E0FC0150
:10437000E85DF84F1082118212821382FC01E8512D
:10438000F84F10821182128213821D920496803C93
:10439000910569F70895EF92FF920F931F93CF93C2
:1043A000DF93EC012396CE010E944C16882309F47A
:1043B00007C1CE0162EE76E040E327E231E00E94E1
:1043C0000D41882311F00E94AF21CE0162EE76E00C
:1043D00040E32BE231E00E940D41882309F44CC0F8
:1043E00082EE96E00E94ED07181619060CF044C004
:1043F0002DB73EB7285030400FB6F8943EBF0FBEE1
:104400002DBFEDB7FEB7319603E117E0ADB7BEB7EC
:1044100012961C930E93119787E393E09383828304
:1044200080E790E09583848384E190E0978386839E
:104430000E94093B0F900F900F900F90EDB7FEB7C1
:10444000128301838AE293E0948383830E94093B71
:104450000F900F900F900F908091190790911A076D
:104460002091170730911807821B930B61E140E000
:104470000E94ED350E943C28CE0162EE76E040E3DA
:104480002FE231E00E940D41882399F08091E206ED
:10449000813339F48091FB0880FD0BC00E94B22D5E
:1044A00008C0803331F48091FB0880FF02C00E9475
:1044B000A82DCE0162EE76E040E322E331E00E94D7
:1044C0000D418823E9F08091E206813351F4809117
:1044D000FB0884FD15C00E94AF218091FB0880611C
:1044E0000BC0803369F48091FB0884FF09C00E94EF
:1044F000AF218091FB088F7E8093FB080E94E42C03
:10450000CE0162EE76E040E325E331E00E940D410A
:10451000882351F182EE96E00E94ED07EC01181617
:104520001906F4F40E946E467B018C01BE018827B7
:1045300077FD8095982F20E13EE040E050E00E941A
:104540001857E60EF71E081F191FE0920B09F0928C
:104550000C0900930D0910930E090E949E2D04C0B2
:10456000009771F50E948C2D2DB73EB72850304032
:104570000FB6F8943EBF0FBE2DBFEDB7FEB7319614
:1045800083E197E0ADB7BEB712969C938E931197D7
:104590008DE193E09383828380E790E09583848329
:1045A00082E791E0978386830E94093B81E0EDB723
:1045B000FEB738960FB6F894FEBF0FBEEDBF01C030
:1045C00080E0DF91CF911F910F91FF90EF900895C0
:1045D000BF92CF92DF92EF92FF920F931F93DF93E0
:1045E000CF9300D0CDB7DEB77C018C010D5F1F4F9C
:1045F000C8010E945941C8010E944C16882309F441
:10460000A0C01A83098327E630E0E20EF31E0DC036
:10461000C80168E371E043E050E00E945F08009742
:1046200079F00F5F1F4F1A83098309811A81D8011E
:104630008C91882309F485C00E151F0548F381C0AD
:104640000D5F1F4F1A8309830E94AF21FF2400E0F2
:1046500014E0EE246E010894C11CD11C5EEFB52E4F
:1046600037C0C6010E942F0CF999FECF1FBA12BDA8
:1046700001BD90BD0FB6F894FA9AF99A0FBEF99958
:10468000FECF1FBA0F5F1F4F12BD01BD015010407A
:1046900080BD0FB6F894FA9AF99A0FBE0097A9F068
:1046A0002F2D30E0F901EE0FFF1FEE0FFF1FE85135
:1046B000F84FA0E0B0E080839183A283B3832855B4
:1046C000374FF901B082EE24E394F3940E5F1F4F4D
:1046D0008091FE08F81608F4C4CFEE2031F00E9455
:1046E0006E4640913D020E9482092DB73EB7285088
:1046F00030400FB6F8943EBF0FBE2DBFEDB7FEB7EA
:10470000319683E197E0ADB7BEB712969C938E9336
:10471000119789E497E09383828380E790E0958303
:10472000848382E791E0978386830E94093B81E03E
:10473000EDB7FEB738960FB6F894FEBF0FBEEDBFCB
:1047400001C080E00F900F90CF91DF911F910F91EA
:10475000FF90EF90DF90CF90BF900895EF92FF927F
:104760000F931F939B01AC018091D8089091D908B9
:10477000A091DA08B091DB080097A105B10549F4D2
:104780002093D8083093D9084093DA085093DB0877
:1047900054C079018A01E81AF90A0A0B1B0BD801E7
:1047A000C701CD97A105B10508F447C02093D808EB
:1047B0003093D9084093DA085093DB0889E599E0F3
:1047C0000E94C7370E949A517B018C010E9485424A
:1047D0000E94143889E599E00E94883A882361F4A0
:1047E0000E949A516E197F09800B910B683C7105EC
:1047F0008105910558F319C08091FC088F70809352
:10480000FC088091FC0882958F7090E00397ACF0D3
:1048100080912F02882389F060915C0370915D0381
:104820008AE791E00E94BC3008C08091FC08982F74
:10483000907F905F8F70892BE2CF1F910F91FF9037
:10484000EF900895EF92FF920F931F939B01AC019D
:104850008091DB01882309F443C08091FC08829594
:104860008F7009F03DC08091FB0883FD39C08091B5
:104870001B0790911C07A0911D07B0911E07009780
:10488000A105B10569F079018A01E81AF90A0A0B54
:104890001B0BD801C70181589145A140B04000F1E0
:1048A00020931B0730931C0740931D0750931E074E
:1048B0008BED9AE061E00E943D2A0E94F50B7B019E
:1048C0008C01611571058105910551F00E944146E9
:1048D0008091FB0885FF04C0C801B7010E944F34D6
:1048E0001F910F91FF90EF9008950E94AF2F0E94AB
:1048F0000E2E0E94270A9091280280E0209121022A
:10490000820F911D90935D0380935C036CE370E0D4
:1049100080E090E00E9438468091FB0885FD03C04E
:1049200080E090E002C08FE694E30E94E14664EFED
:1049300071E080E090E00E94A85180E00E94652F25
:1049400088EF9AE061E00E943D2A87ED99E060E0FF
:104950000E94664C882329F48091FB088064809330
:10496000FB088AEE9AE061E00E943D2A60915C03B8
:1049700070915D038AE791E00E94BC30882321F0AA
:104980008091FC088F7004C08091FC088F7080615A
:104990008093FC0864EF71E080E090E00E94A851F1
:1049A0000E94432D089582E00E94AE29282F30E016
:1049B00086FF41C02F7030702230310591F02430D5
:1049C000310509F121303105B1F587FF03C00E949F
:1049D000B22D08956091CD027091CE0281E599E0EB
:1049E00009C087FF03C00E94A82D089589E599E0BA
:1049F00060E070E00E949C2C60ED77E080E090E049
:104A00000E94A851089587FF06C081E00E94AE2948
:104A10000E943C2808952091FC08822F8F7090E01E
:104A20006091FD08019670E00E9457578F70207FBB
:104A3000282B2093FC0808952F923F924F925F926B
:104A40006F927F928F929F92AF92BF92CF92DF929E
:104A5000EF92FF920F931F93DF93CF93CDB7DEB703
:104A6000AA970FB6F894DEBF0FBECDBF20913D02CE
:104A70002C8B30914B023B8B0E9485420E94143854
:104A80009093DD088093DC08009721F0825A9C4FB8
:104A90000E9418130E94D3240E946E465B016C0191
:104AA0008091E2089091E308A091E408B091E508B4
:104AB0008A159B05AC05BD0509F4B0C2A092E208B9
:104AC000B092E308C092E408D092E50880E00E942A
:104AD000652F8091FB0820910B0930910C094091C2
:104AE0000D0950910E0981FF08C0A216B306C40635
:104AF000D50650F00E948C2D07C0A216B306C4063E
:104B0000D50610F40E949E2D0E94F7298091FB0883
:104B100084FDC4C083FF04C04C89442309F0BEC097
:104B2000C601B5012CE330E040E050E00E946A5736
:104B300079018A018091DE089091DF08A091E00858
:104B4000B091E108E816F9060A071B0709F4A6C0A8
:104B5000E092DE08F092DF080093E0081093E1088D
:104B6000662410E09B89892F90E09AA789A78AC0C4
:104B7000862DBE016F5F7F4F0E94B519CE01019651
:104B8000B601A5010E940519882309F47AC0298578
:104B90003A852115310509F474C0A091FD08AE8B4A
:104BA00077241A8A190144245524B62DBF5FB8A76B
:104BB00053C08A89880DE82EFF24C7010196E9A514
:104BC000FAA5E817F907E1F1ACA1BDA18C9190E03D
:104BD000082C02C0959587950A94E2F780FD30C0B5
:104BE000EEA1FFA1808190E0082C02C095958795E9
:104BF0000A94E2F780FF24C08701000F111F000F05
:104C0000111F0851184F60916E0270E080E090E033
:104C1000A20191010E94185724E630E040E050E0E4
:104C20000E946A57D8012D933D934D935C9313973F
:104C3000E8EAF8E0EE0EFF1EE8A5D701EC9311E0DC
:104C40000894811C911CF8E08F16910409F0B1CFF3
:104C500073942A89285F2A8B3E89731690F4872DD6
:104C600090E088249924AC014150574F5DA34CA398
:104C7000ABE0B0E0AC0FBD1FA80FB91FBFA3AEA340
:104C800098CF639480911F07681608F471CF1123A1
:104C900029F0C601B5014C890E9482098091FB0868
:104CA00083FF50C14424FB89EF2FF0E0FC8FEB8F92
:104CB0002B8921502D8F30E0C901880F991F880F53
:104CC000991FAC01485D584F5F8F4E8FDC01A85192
:104CD000B84FB9A3A8A3F901E855F74FFBA3EAA37E
:104CE00014C1842D90E0FC01E150F74F2081F42D98
:104CF000FF0FFF0FFF0FFD8B66247724422F50E03C
:104D0000588F4F8BDC01AB5FB64FBA8FA98F5D8890
:104D1000560C852C992498EAE92E98E0F92EE80C97
:104D2000F91CF7018081882309F44DC08401000F2C
:104D3000111F000F111FF801E851F84F8081918178
:104D4000A281B381A816B906CA06DB06E0F1852D5B
:104D500060E00E94A828C40101962B8D3C8D281785
:104D60003907D1F050922007D7018C918093210709
:104D7000085D184FF801808191819501281B390B3E
:104D80003093230720932207A0922407B09225078F
:104D9000C0922607D0922707F401EE0FFF1FEE0FF7
:104DA000FF1FDF01A85DB84F1D921D921D921C923E
:104DB0001397E851F84F1082118212821382F40186
:104DC000E855F74F10828F89988D062C02C0959573
:104DD00087950A94E2F780FD8FC09401220F331F5C
:104DE000220F331F8901085D184FF80180819181DE
:104DF000A281B381A816B906CA06DB0608F47CC0F6
:104E0000F8EE2F2EF7E03F2E220E331EF1018081A7
:104E10009181A281B381A816B906CA06DB0608F003
:104E20006BC0852D61E00E94A828FB89FF2309F44F
:104E300063C0C40101962B8D3C8D2817390709F4F6
:104E40005BC0A98DBA8D8C9190E0062C02C095951F
:104E500087950A94E2F780FF4FC0BC89BB2309F411
:104E60004BC08091FB0884FD47C080915202F8013D
:104E70002081318142815381280F311D411D511DF7
:104E8000AE8DBF8D2D933D934D935C931397809181
:104E90005902E82EFF2400E010E084EC9FEFAFEF12
:104EA000BFEFE80EF91E0A1F1B1FF10180819181DF
:104EB000A281B381E80EF91E0A1F1B1FA8A1B9A188
:104EC000ED92FD920D931C931397E8EAF8E08E0E95
:104ED0009F1ED4018C91EAA1FBA18083A216B30688
:104EE000C406D50648F0AE14BF04C006D10620F4AF
:104EF0008D8D61E00E94A8280894611C711CF8E067
:104F00006F16710409F003CF43948091FD08481691
:104F100008F4E7CE0E94432D3091FE08E8EEF7E05A
:104F200020E00DC081919191A191B1910197A109CA
:104F3000B1098E5F9F4FAF4FBF4F20F02F5F2317F8
:104F400088F361C05B89552369F08091FB0884FF79
:104F500009C01091FE0840E021E030E08B89682F05
:104F600070E02EC09C899923A1F331C0842F90E07A
:104F70006217730711F1DC01E3E0B695A795EA9596
:104F8000E1F7542F5770FD01E150F74F808190E019
:104F9000052E02C0959587950A94E2F780FF0DC013
:104FA000AB5FB64F8C9190E002C0959587955A956E
:104FB000E2F780FF02C061E006C04F5F2F5F3F4F06
:104FC0004117A0F260E08B8981500E94A8280E94BE
:104FD000432DC601B50123E030E040E050E00E94DF
:104FE0006A579B01AC012F5F3C4F81E0D9016C9166
:104FF0000E94122CC601B5010E94AE23C601B50164
:105000000E9422240BC00E94CC288091FB08877F3D
:105010008093FB08B0914B02BB8B94CFAA960FB63E
:10502000F894DEBF0FBECDBFCF91DF911F910F91DE
:10503000FF90EF90DF90CF90BF90AF909F908F90B8
:105040007F906F905F904F903F902F9008959C01BC
:10505000F999FECF32BD21BDF89A80B508959C0123
:10506000F999FECF1FBA32BD21BD60BD0FB6F894CD
:10507000FA9AF99A0FBE0895E0910F09F09110097C
:1050800009950895DB01482F50E0405F5F4F84E0B1
:10509000440F551F8A95E1F750961C92509720E0D7
:1050A00030E0F999FECFC901840F951F92BD81BDF3
:1050B000F89A80B5FD01E20FF31F8083882331F059
:1050C0002F30310519F02F5F3F4FEBCF0895DB01F3
:1050D000482F50E0405F5F4F94E0440F551F9A9572
:1050E000E1F750961C92509720E030E0FD01E20F6E
:1050F000F31FE081F999FECF1FBAC901840F951FF4
:1051000092BD81BDE0BD0FB6F894FA9AF99A0FBE30
:10511000EE2331F02F30310519F02F5F3F4FE6CFEE
:10512000089580E694E0FC01EB55FB4FE081F9998E
:10513000FECF1FBA92BD81BDE0BD0FB6F894FA9ABA
:10514000F99A0FBE019624E08636920761F708951A
:10515000282F277086958695869590E0662369F0BE
:10516000FC01E150F74F81E090E002C0880F991FE9
:105170002A95E2F72081282B0DC0FC01E150F74F62
:1051800081E090E002C0880F991F2A95E2F7809590
:1051900020812823208308951092FF08109200098F
:1051A0001092010910920209109203091092040949
:1051B0000895EDECF1E020E030E0F999FECF32BD4A
:1051C00021BDF89A80B580832F5F3F4F37962232FA
:1051D000310599F7809136028F5F8093FD0890E04A
:1051E00023E0880F991F2A95E1F78093FE08089520
:1051F000E4EBF2E081E290E02081F999FECF1FBA62
:1052000092BD81BD20BD0FB6F894FA9AF99A0FBEEF
:10521000019737972FEF8F3F920771F780913602F2
:105220008F5F8093FD0890E033E0880F991F3A95D7
:10523000E1F78093FE080895AC01FB010FC0F999D6
:10524000FECF1FBADA01A80FB11DB2BDA1BD20BDAE
:105250000FB6F894FA9AF99A0FBE31968E2F861BE4
:105260002081222361F7F999FECF1FBA480F511D03
:1052700052BD41BD10BC0FB6F894FA9AF99A0FBE10
:105280000895582F282F392FF9018E2F851BF99952
:10529000FECF90E0805C9F4F92BD81BDF89A80B5B3
:1052A0009081882331F0992349F0891739F4319698
:1052B000ECCF80E0992319F481E0089580E008950F
:1052C0001092E9081092E80888E193E09093E708CB
:1052D0008093E6080895EF92FF920F931F93CF9368
:1052E000DF93E82E162F042FF22E662321F0623072
:1052F00081F4222371F08E2D0E945053892B11F0DE
:1053000000E024C0FF2011F480E001C080E8082BF9
:105310001DC0C0E0D0E08E2D0E945053892B81F437
:10532000113031F0123061F483E0C032D80744F418
:1053300061E070E080E090E00E94A8512196EBCF00
:10534000FF2019F4C052D3400CF00068802FDF9189
:10535000CF911F910F91FF90EF9008950F931F939E
:10536000082F10911109107861E070E080E090E062
:105370000E94A8518FE10E945053892B21F48FE1A4
:10538000602F41E013C08EE10E945053892B21F41D
:105390008EE1602F42E00AC08DE10E945053892BBC
:1053A00011F040E007C08DE1602F44E0212F0E9402
:1053B0006B29482F8091110990E08F709070242FF5
:1053C00030E0892B39F42F703070232B71F0842F4B
:1053D000806406C02F703070232B39F4842F8062D4
:1053E000409311091F910F910895842FF9CF8BE0FD
:1053F0000E94505340E02091670230E082179307EB
:1054000009F041E0440F440F8091FB088B7F842B0F
:105410008093FB080895EF92FF920F931F938C01E6
:1054200046EEE42E48E0F42E6AE070E00E94575702
:10543000C7014AE050E00E941456C8016AE070E0DB
:105440000E945757BC01C7014AE050E00E94145621
:105450001F910F91FF90EF900895CF93DF93EC0190
:1054600004C086EE98E00E945455FE012196649196
:105470006623B9F7DF91CF9108950F931F93CF93D0
:10548000DF938C01462F86EE98E060E00E9419328F
:10549000E80104C086EE98E00E9454559E01201B4E
:1054A000822FFE01219664916623A1F7992787FD3B
:1054B0009095C0E1D0E0C81BD90B05C08FED9DE0F1
:1054C0000E942D2A2197D7FFF9CFDF91CF911F910D
:1054D0000F910895EF92FF920F931F93CF93DF9355
:1054E0007C018C01F3E0000F111FFA95E1F7081B16
:1054F000190B03531E4FF8018281938160E00E94D3
:105500003D2A8CEA9DE061E00E943D2A86EE98E00B
:1055100060E041E00E941932F801868180FF05C0F9
:1055200086EE98E00E94FD3104C086EE98E00E946D
:105530000732F3E1EF16F10409F45EC084E1E816E6
:10554000F10454F4E1E0EE16F104B1F0FCE0EF16E2
:10555000F10409F08CC065C08BE1E816F10409F490
:105560006AC0ECE1EE16F10409F475C0F4E1EF163F
:10557000F10409F07CC047C08091D401C82FD0E06D
:10558000E097D7FD05C08AEA9DE00E942D2A07C05A
:1055900088EA9DE00E942D2AD095C195DF4FCE016B
:1055A00064E070E00E94575786EE98E04AE050E0D1
:1055B0000E94145686EA9DE00E942D2ACE0164E0E6
:1055C00070E00E945757BC01E4E0660F771FEA9530
:1055D000E1F7681B790B29F483EA9DE00E942D2AEC
:1055E00006C086EE98E04AE050E00E9414568EE92C
:1055F0009DE00E942D2A61C08CE99DE00E942D2A29
:105600006091520220C0809159028C3320F08AE9C7
:105610009DE00E942D2A6091590270E06C53704009
:1056200007C07091280260E080912102680F711D0F
:1056300086EE98E00BC060918A028DE070E00E94D7
:105640005D5260918A0286EE98E070E04AE050E098
:105650000E94145632C0809191026FEF70E0681B77
:1056600071098CE00E945D5260919102ECCFF701CC
:1056700053E0EE0FFF1F5A95E1F7EE19FF09E353D0
:10568000FE4F81816081813051F4662319F483E9F2
:105690009DE002C086E99DE00E942D2A07C086EEAB
:1056A00098E070E04AE050E00E94145687E1E81666
:1056B000F10419F481E99DE011C0C70143970297F5
:1056C00020F0E8E1EE16F10419F48CE89DE006C044
:1056D000F1E1EF16F10421F487E89DE00E942D2A04
:1056E000DF91CF911F910F91FF90EF900895EF926E
:1056F000FF920F931F93182F092F0E946A2A212FC0
:10570000302FC9018C018AEAE82E82E00E94AE297E
:10571000482F282F30E0C9018F709070823091059A
:10572000D9F08430910561F1019709F068C0F80162
:10573000B3E0EE0FFF1FBA95E1F7E01BF10BE35367
:10574000FE4F868180FF5EC090818181891709F4B8
:1057500059C09F5F908356C0F801A3E0EE0FFF1F72
:10576000AA95E1F7E01BF10BE353FE4F868180FF22
:1057700046C08081882309F442C0815080833FC0A5
:1057800046FF3DC047FF0BC08091B402882311F053
:10579000E092B4020E94F828FF24F39434C003304E
:1057A000110541F48091E201882309F1FF240CE006
:1057B00010E029C00C30110521F4FF240EE010E0A8
:1057C00022C00531110541F480916002882379F4EB
:1057D000FF2407E110E017C00231110541F4809168
:1057E0004B02882321F4FF2405E110E00CC0C8011E
:1057F000019662E270E00E9457578C0103C0442377
:1058000009F483CFFF24C8010E946A2AFF2009F40B
:105810007CCF86EE98E00E9407321F910F91FF9097
:10582000EF9008950F931F93CF93DF93482F062F88
:1058300086EE98E060E00E9419328091FC088F703B
:1058400019F48EEC9DE010C08CEC9DE00E942D2A96
:105850006091FC086F7086EE98E070E04AE050E0DE
:105860000E9414568AEC9DE00E942D2A8091FB082C
:1058700080FD03C08EEB9DE00AC081FD06C082FF63
:105880000AC080916002882331F082EB9DE061E0E4
:105890000E943D2A26C0E091FC08EF70F0E0E15044
:1058A000F74F1081C1E0D0E08091FC088F7051F477
:1058B00080914B0290E0C817D90721F410FD06C073
:1058C0006DE405C010FD02C06FE501C0602F86EEDB
:1058D00098E00E9454552196C930D10511F01695D3
:1058E000E3CF8DEA9DE00E942D2A86EE98E06EE0DF
:1058F00041E00E94193260E08091FC0882958F702F
:1059000090E003970CF061E086EE98E00E94CB31C6
:1059100086EE98E06FE041E00E9419328091FB082A
:1059200086FF05C086EE98E062E00E94CB31DF91F1
:10593000CF911F910F910895EF92FF920F931F93B4
:10594000CF93DF938C017B0186EE98E00E94483272
:1059500086EE98E060E040E00E941932C0E0D0E0BE
:10596000F801EC0FFD1F608186EE98E070E04AE0E0
:1059700050E00E94145684ED9DE00E942D2A21964D
:10598000C330D10569F7F801638186EE98E070E0D5
:105990004AE050E00E94145686EE98E060E041E054
:1059A0000E94193282ED9DE00E942D2A86EE98E039
:1059B000B7014AE050E00E941456DF91CF911F9149
:1059C0000F91FF90EF9008952091FB082170F999B5
:1059D000FECF1FBA80E390E092BD81BD20BD0FB61F
:1059E000F894FA9AF99A0FBE2091FB08229521703B
:1059F000F999FECF1FBA81E390E092BD81BD20BD31
:105A00000FB6F894FA9AF99A0FBE40910B0950918B
:105A10000C0960910D0970910E0982E390E02FE26C
:105A200038E20E94CB080895F999FECF80E390E018
:105A300092BD81BDF89A90B591708091FB088E7FE0
:105A4000892B8093FB08F999FECF81E390E092BD0A
:105A500081BDF89A90B591709295907F8091FB08E6
:105A60008F7E892B8093FB0882E390E067E278E2E7
:105A70000E94890860930B0970930C0980930D09AB
:105A800090930E090895EF92FF920F931F93CF9377
:105A9000DF9383E060E00E94FC5204E019E0909103
:105AA000FB0890FF0BC091FD09C080916002882324
:105AB00011F092FD03C0F801608101C060E0C7E011
:105AC000D0E0E62EFF2486E160E00E94FC52B701A0
:105AD0000C2E02C0759567950A94E2F7617085E116
:105AE0000E94FC5286E161E00E94FC522197FFEF88
:105AF000CF3FDF0741F70150104088E00E3F180705
:105B000071F683E061E00E94FC52DF91CF911F911A
:105B10000F91FF90EF9008958091FB088D7F809307
:105B2000FB0810920B0910920C0910920D091092AB
:105B30000E090E94E42C0E94432D08958091FB08D9
:105B400082608093FB080E94E42C0E94432D0895FC
:105B50008091FB088E7F8093FB080E94432D0E945A
:105B6000E42C08958091FB0881608093FB080E94DB
:105B7000432D0E94E42C0895AF92BF92CF92DF9202
:105B8000FF920F931F93CF93DF935B016C01FF2470
:105B9000C1E0D0E03CC086EE98E00E94483286EE3C
:105BA00098E060E040E00E9419320F2D10E0B8014B
:105BB0006F5F7F4F86EE98E04AE050E00E941456F7
:105BC0001092FF0810920009109201091092020928
:105BD000109203091092040993E0169507959A957F
:105BE000E1F70150174F8F2D87709E0102C0220FE1
:105BF000331F8A95E2F7C901F8012081282B208301
:105C00000E94432DC601B5010E94A851F3948091D2
:105C1000FE08F81608F4BFCFFF24FBCF64EF71E055
:105C200080E090E00E94A851F999FECF12BC11BC0F
:105C3000F89A90B5943620F48AE0989F902D11241C
:105C40009B3C59F4F999FECF81E290E092BD81BD71
:105C5000F89A80B58A3A09F091C00E94F8280E940B
:105C6000E42C80E490E06CE371E00E941C2980E663
:105C700090E065E471E00E941C2980E890E06FE408
:105C800071E00E941C2981E29EE060E00E943D2AB2
:105C900082E19EE061E00E943D2A80E091E0F99976
:105CA000FECF1FBA92BD81BD10BC0FB6F894FA9A10
:105CB000F99A0FBE019628E08030920781F720E024
:105CC00031E0E1E0F0E043E5F999FECF1FBA32BDE3
:105CD00021BD40BD0FB6F894FA9AF99A0FBEF99912
:105CE000FECF1FBA2F5F3F4F32BD21BD2150304044
:105CF000CF016AE070E00E945757605D60BD0FB64B
:105D0000F894FA9AF99A0FBEF999FECF1FBA2E5F4E
:105D10003F4F32BD21BDCF016AE070E00E9457576E
:105D2000805D80BD0FB6F894FA9AF99A0FBE225F93
:105D30003F4F84E02030380711F03196C5CF80E620
:105D400094E02FEFF999FECF1FBA92BD81BD20BD1F
:105D50000FB6F894FA9AF99A0FBE019634E0863697
:105D6000930781F764EF71E080E090E00E94A85112
:105D7000E0910F09F0911009099516C00E94D928E9
:105D800020E634E0F999FECF32BD21BDF89A80B506
:105D9000F901EB55FB4F80832F5F3F4F84E02636A0
:105DA000380781F70E94142D80E00E94AE2990E010
:105DB0008F7090708230910521F18430910521F12E
:105DC000019709F04CC064E670E080E090E00E942A
:105DD000A8518DE10E945053892B29F460E273E0B1
:105DE00080E090E00BC06091750270E080E090E090
:105DF00028EE33E040E050E00E9418570E94BC2D8E
:105E00002EC081E290E020C082E09EE060E00E942F
:105E10003D2A60ED77E080E090E00E94A85181EF9C
:105E20009DE060E00E943D2A81EE9DE061E00E94DD
:105E30003D2A80E00E94AE2986FFFBCF86EE98E0E7
:105E40000E94483280E090E00E94772B8091B4025B
:105E5000882329F0E0910F09F091100909958CE051
:105E600061E00E94BD528DE061E00E94BD526091F0
:105E70008A028DE070E00E945D52809191026FEF86
:105E800070E0681B71098CE00E945D520895DF93F9
:105E9000CF93CDB7DEB727970FB6F894DEBF0FBE0E
:105EA000CDBFCE0101960E94D0338C8190E0059643
:105EB00067E070E00E94575727960FB6F894DEBF50
:105EC0000FBECDBFCF91DF910895DF92EF92FF9289
:105ED0000F931F93D82E0E946E467B018C0186EE95
:105EE00098E060E04D2D0E941932C801B7010E9470
:105EF0005B450E940B2A8DED9DE00E942D2AC80172
:105F0000B7010E9455450E940B2A8AED9DE00E9430
:105F10002D2A0E94472FE82FF0E0EE0FFF1FE554D7
:105F2000FD4F808191810E942D2A88ED9DE00E9485
:105F30002D2AC801B7010E9443450E940B2A86ED15
:105F40009DE00E942D2AC801B7010E944F450E9482
:105F50000B2A1F910F91FF90EF90DF9008958F9281
:105F6000AF92CF92EF920F931F93DF93CF93CDB762
:105F7000DEB760970FB6F894DEBF0FBECDBF83E0EB
:105F800061E00E94BD5281E061E00E94BD5286E165
:105F900061E00E94BD5285E161E00E94BD5283E054
:105FA00061E00E94FC5281E061E00E94FC5210928C
:105FB000FF08109200091092010910920209109234
:105FC0000309109204090E94432D81E060E00E94C1
:105FD000FC5280E061E00E94BD5280E061E00E94DE
:105FE000FC5287ED99E060E00E94024711E01093B7
:105FF00081008CE061E00E94BD528DE061E00E9472
:10600000BD5260918A028DE070E00E945D528091E5
:1060100091026FEF70E0681B71098CE00E945D5285
:1060200000D000D0EDB7FEB73196ADB7BEB7119630
:106030001C9211821282138286EE98E061E043E1A5
:106040002FEF02E1E4E1EE2E75E1C72E56E1A52E19
:1060500037E1832E0E94BF320F900F900F900F9068
:1060600086EE98E060E142E020E00E9450328BE052
:1060700060E00E94BD528BE061E00E94FC5289E723
:106080009CE00E94DF4E8091FB08816081788093C4
:10609000FB081092FC081093FD0888E08093FE082E
:1060A00010920B0910920C0910920D0910920E0912
:1060B000DE011196ECE0F3E001900D928150E1F7E2
:1060C000DE011996E4E0F3E088E001900D92815042
:1060D000E1F786EE98E061E08E010F5F1F4FA801A7
:1060E0000E94D5311A821B8281E08C8386EE98E073
:1060F00060E0A8010E94D53186EE98E062E0AE0132
:10610000475F5F4F0E94D5318CE161E00E94BD5234
:106110008CE160E00E94FC528FE160E00E94BD5281
:106120008EE160E00E94BD528DE160E00E94BD52B0
:106130008FE161E00E94FC528EE161E00E94FC521E
:106140008DE161E00E94FC520E949D33882329F476
:106150008091FB0880628093FB0860960FB6F894EC
:10616000DEBF0FBECDBFCF91DF911F910F91EF909A
:10617000CF90AF908F9008950F931F93DF93CF939D
:10618000CDB7DEB728970FB6F894DEBF0FBECDBFF0
:10619000FC018B0180918302858384E893E0BF0139
:1061A00044E00E94C63A882311F490E032C0109374
:1061B000CE020093CD028091E201882319F00E9463
:1061C000D84021C08091E90189838091F0018A83C0
:1061D0008091F7018B838091FE018C838091050271
:1061E0008D8380910C028E83809113028F83809126
:1061F0001A028887CE010196BE016B5F7F4F40E097
:1062000050E00E94A33A90E0882309F491E081E0F5
:106210009827892F28960FB6F894DEBF0FBECDBF02
:10622000CF91DF911F910F9108950F931F938C01D0
:10623000FC01868160E00E94FC5281E090E00E94B7
:106240001852F801868161E00E94FC5281E090E0E2
:106250000E941852F801868160E00E94FC5284E698
:1062600090E00E9418521F910F910895CF92DF92F3
:10627000EF92FF920F931F93CF93DF93D82EC92EE7
:10628000282F392FC9018C01C0E0D0E0E62EFF2471
:10629000F801878161E00E94BD52B7010C2E02C057
:1062A000759567950A94E2F76170F80187810E94FD
:1062B000FC5221960F5F1F4FC830D10549F78D2D35
:1062C0009C2D0E941531DF91CF911F910F91FF906E
:1062D000EF90DF90CF900895CF92DF92EF92FF92F0
:1062E0000F931F93CF93DF93D82EC92E282F392FCA
:1062F000C9018C01C0E0D0E0E62EFF24F8018781BF
:1063000061E00E94BD52B7010C2E02C075956795E1
:106310000A94E2F76170F80187810E94FC5221968D
:106320000F5F1F4FC430D10549F78D2D9C2D0E9462
:106330001531DF91CF911F910F91FF90EF90DF907A
:10634000CF9008951F93CF93DF93EC01162F8C818C
:10635000642F0E94FC528D818F3F19F060E00E94F3
:10636000FC528F8584FF05C0CE01612F0E9436311B
:106370000EC0612F70E084E0759567958A95E1F70E
:10638000CE010E946C31CE01612F0E946C31DF91F1
:10639000CF911F91089541E00E94A23181E090E0E9
:1063A000089540E00E94A2310895EF92FF920F936A
:1063B0001F93CF93DF938C017A016770660F660F8E
:1063C000660F60640E94D131C0E0D0E0D801ED9149
:1063D000FC91D701AC0FBD1F0190F081E02DC801E9
:1063E0006C9109952196C830D10581F7DF91CF9145
:1063F0001F910F91FF90EF900895FC016089862F07
:106400008160808B6960CF010E94D1310895FC01C9
:1064100060896E7F608B68600E94D1310895FC01B5
:106420006089862F8460808B6C60CF010E94D1319F
:106430000895DF93CF93CDB7DEB728970FB6F894C2
:10644000DEBF0FBECDBF9C01FE013196ACE1B3E0D3
:1064500088E00D9001928150E1F7F9018389481796
:1064600010F0482F4150E42FF0E0EE0FFF1FEC0F2B
:10647000FD1F8181680F6068C9010E94D131289693
:106480000FB6F894DEBF0FBECDBFCF91DF91089558
:1064900061E00E94D13180ED97E00E94185208958A
:1064A000CF93DF93EC01423018F08F8588608F879F
:1064B0004B8B1C8A222329F0413019F48F8584608C
:1064C0008F8780E593EC0E9418528C8160E00E94D7
:1064D000FC528E8160E00E94FC528D818F3F19F04A
:1064E00060E00E94FC526F8564FD1DC0CE0163E038
:1064F0000E946C3184E991E10E941852CE0163E060
:106500000E946C3184E991E10E941852CE0163E04F
:106510000E946C3186E990E00E941852CE0162E040
:106520000E946C3116C06062CE010E94D13184E9B4
:1065300091E10E9418526F856062CE010E94D131B4
:1065400086E990E00E9418526F856062CE010E9439
:10655000D1316F856062CE010E94D13184E0888B99
:10656000CE010E940F32CE010E94483282E0898B18
:10657000CE0166E00E94D131DF91CF9108956F92F4
:106580007F928F92AF92CF92EF920F931F93DF93F0
:10659000CF93CDB7DEB73C01162F842FF301448390
:1065A00025830683E782C086A18682869D859387A0
:1065B0009E8594879F8595879889968761E00E943C
:1065C000BD52F30185818F3F19F061E00E94BD52F9
:1065D000F301868161E00E94BD52112319F0F3019D
:1065E000178603C080E1F3018787C30160E141E0C2
:1065F00020E00E945032CF91DF911F910F91EF90D8
:10660000CF90AF908F907F906F900895482F6AE061
:106610000E943757282F30E084E0220F331F8A95DD
:10662000E1F7842F0E943757892F820F0895CF9367
:10663000DF93EC018091120990911309883691053E
:1066400059F589E79CE068E670E00E94054E89E70D
:106650009CE060E00E94874E88810E940633682F8C
:1066600070E06F77707089E79CE00E94874E8981A7
:106670000E940633682F89E79CE00E94874E8A813A
:106680000E940633682F89E79CE00E94874E8B8129
:106690000E940633682F2DC08F36910509F04AC03D
:1066A00089E79CE06FE670E00E94054E89E79CE078
:1066B00060E00E94874E88810E940633682F6068E0
:1066C00089E79CE00E94874E89810E940633682FEB
:1066D00089E79CE00E94874E8A810E940633682FDA
:1066E00089E79CE00E94874E8B810E940633682FC9
:1066F000686089E79CE00E94874E8C810E94063387
:10670000682F89E79CE00E94874E8D810E940633A6
:10671000682F89E79CE00E94874E8E818E510E94EF
:106720000633682F89E79CE00E94874E89E79CE04A
:106730000E94CA4EDF91CF91089588E690E0909331
:1067400013098093120989E79CE068E670E00E94D3
:10675000054E89E79CE060E00E94874E89E79CE057
:106760000E94CA4E8823D9F08FE690E090931309D7
:106770008093120989E79CE06FE670E00E94054E65
:1067800089E79CE060E00E94874E89E79CE00E94D8
:10679000CA4E882321F0109213091092120908950D
:1067A0001F93CF93DF93EC0160911209709113094D
:1067B0006115710509F46FC089E79CE00E94054EE0
:1067C00089E79CE060E00E94874E89E79CE00E9498
:1067D000CA4E609112097091130989E79CE047E065
:1067E00050E00E94DB4E89E79CE00E94184E282F63
:1067F0002F7722952F701AE0219F900111248F701E
:10680000820F888389E79CE00E94184E282F2295EA
:106810002F70219F900111248F70820F898389E747
:106820009CE00E94184E282F2F7322952F70219FD5
:10683000900111248F70820F8A8389E79CE00E9467
:10684000184E87708B8389E79CE00E94184E282F92
:1068500022952F70219F900111248F70820F8C83BD
:1068600089E79CE00E94184E282F22952F70219FC7
:10687000900111248F70820F8D8389E79CE00E9424
:10688000184E282F2F70225E82958F70819FC00135
:106890001124280F2E83DF91CF911F9108950F931C
:1068A0001F93DF93CF93CDB7DEB727970FB6F8943A
:1068B000DEBF0FBECDBF8E010F5F1F4FA8010E942C
:1068C0001244C8010E94173327960FB6F894DEBF12
:1068D0000FBECDBFCF91DF911F910F9108950F9300
:1068E0001F93DF93CF93CDB7DEB727970FB6F894FA
:1068F000DEBF0FBECDBF8E010F5F1F4FC8010E94CC
:10690000D033C8010E94614527960FB6F894DEBFC8
:106910000FBECDBFCF91DF911F910F91089589E7F1
:106920009CE00E94DF4E0895DF92EF92FF920F935A
:106930001F93CF93DF93D82E862FBA01213041F4D5
:10694000675F7F4F9B0140E050E0695070400EC090
:10695000223029F020E030E040E050E007C06250F3
:1069600070409B0140E050E06E5F7F4FE82EFF24B7
:106970008EE593E0E80EF91E8B01E7010FC0F88168
:10698000E0E0898190E08E2B9F2BA0E0B0E0280F03
:10699000391F4A1F5B1F229602501040023011051A
:1069A00070F7CB018E7FD701A80FB91F6817790741
:1069B00079F08C9190E0A0E0B0E0BA2FA92F982F49
:1069C000882702C040E050E0280F391F4A1F5B1F94
:1069D000CA01AA27BB270097A105B10599F7C901EC
:1069E00080959095ED2DF0E0E25AFC4F90838183E5
:1069F000DF91CF911F910F91FF90EF90DF9008955D
:106A0000109276031092770380E4809372031092C1
:106A100073038093740388E16EE044E150E020E06A
:106A20000E9494340895282F662321F080918303D7
:106A30008617E1F4809184038823C1F48091850353
:106A40008833A1F4809181038B3781F4E22FF92FF1
:106A50008091B00383838091B10382838091B203DC
:106A600081838091B303808381E0089580E008955D
:106A70000F931F93BC010EE513E0C8010E949C41D7
:106A8000C80106966BE479E00E949C411F910F912A
:106A90000895EF92FF920F931F937B010E94383568
:106AA0000CE713E0C801B7010E94A441C801049794
:106AB00061E579E00E94A4411F910F91FF90EF9052
:106AC0000895EF92FF920F931F93CF93DF937C0172
:106AD000EB018A018FE199E00E9449358881807F2E
:106AE000803E49F088819981AA81BB818F5F9F4F49
:106AF000AF4FBF4F31F48EE593E064E273E00E9444
:106B00009C4188E080936A0310926B038CE693E0CB
:106B10006AE37EE049E050E00E94320810926E0382
:106B200081E1809375031093820300938303F092B5
:106B30008003E092810310928403109286031092E6
:106B40008703DF91CF911F910F91FF90EF900895F0
:106B5000EF92FF920F931F9304E613E0C8010E9487
:106B6000383574E1E72EF12CE00EF11EC80148968D
:106B7000B7010E94A441C70161E579E00E94A441E8
:106B80000E9400351F910F91FF90EF900895BC0176
:106B900081E08093140989E599E00E94A441089559
:106BA0000F931F938C01889690936E0380936F03CD
:106BB0000E9400351092900310929103045E1F4FC3
:106BC00082E36AE1A80122E00E949434C8014A9657
:106BD0000E940E431F910F9108951F93CF93DF934F
:106BE000EC01142F8091270990912809A09129097F
:106BF000B0912A092B2F332744275527209384034C
:106C0000A0938503909386038093870360938D03FD
:106C1000CE010E94D0351123B9F49E0140E050E02E
:106C20008091270990912809A0912909B0912A09FA
:106C3000820F931FA41FB51F8093270990932809E3
:106C4000A0932909B0932A09DF91CF911F9108954C
:106C5000CF93DF939C01862F806180938D036430F6
:106C600029F02115310511F421E030E090918203E3
:106C7000809180038093820390938003909183039B
:106C8000809181038093830390938103C7E8D3E0CD
:106C90008881A901480F511D2C814C832883252F01
:106CA0003327219753E0C338D50791F71D861E86F9
:106CB00080E5898710926E0388E280936F030E94BB
:106CC000A83584E08B871C8682E36AE14CE150E0C2
:106CD00022E00E94943486E390E00E940E43DF910C
:106CE000CF910895809125099091260960E00E9436
:106CF00028368091840390E0A0E0B0E0BA2FA92F5D
:106D0000982F882720918503820F911DA11DB11D09
:106D1000BA2FA92F982F882720918603820F911DC3
:106D2000A11DB11DBA2FA92F982F88272091870365
:106D3000820F911DA11DB11D8093270990932809F1
:106D4000A0932909B0932A090895E82FA0916E0312
:106D5000B0916F03F0918C034091820350E0292F92
:106D600030E04217530709F08EC0809183038E17DD
:106D700009F089C080918D03E82F81FF4EC01092E9
:106D80006E038CE280936F030E94A83582E18093AA
:106D90008D0390918203809180038093820390936E
:106DA0008003909183038091810380938303909368
:106DB0008103E7E8F3E021E030E08081A901480F9A
:106DC000511D44831082252F3327319753E0E33838
:106DD000F50799F715861686118212828091CC02EA
:106DE000838314828D5F8093CC0282E0818B84E068
:106DF000828B95E0938B148A80E68187938788E75E
:106E0000848782E36AE140E250E022E00E94943409
:106E10008AE390E00E940E4336C084FF34C04F2FB7
:106E200050E084E0559547958A95E1F79A2F80E0E8
:106E30002B2F30E0282B392BCA01880F991F880F80
:106E4000991F281B390B2451304037FF02C020E026
:106E500030E03093260920932509232B69F09A010D
:106E6000220F331F220F331F2E5D3F4F685070409B
:106E70006217730740F009C0E0FF05C080E090E0B2
:106E800060E00E94283620E030E0C90108950F93A9
:106E90001F93DF93CF930F92CDB7DEB78C01045EC3
:106EA0001F4F10936E030C511040802F845E80930F
:106EB0006F0389830E940035085F1F4F109384037E
:106EC0008981845180938503085F1F4F88E26AE1BE
:106ED000A80121E00E949434C8014A960E940E4302
:106EE0000F90CF91DF911F910F910895FF920F9313
:106EF0001F939C01F62E8FE199E0B9010E9449355C
:106F00000AE613E088E080936A0310926B03C801DD
:106F100002966AE37EE049E050E00E9432088CE489
:106F200080936F0381E1809375030E940035109276
:106F300082038BE7809383038AE080938003F0923F
:106F400081031092840388E3809385031092860363
:106F500010928703025E1F4F80E3F80111928A9519
:106F6000E9F7C80161EF7EE04AE050E00E94320894
:106F700088E26AE140E450E021E00E9494348AE52E
:106F800090E00E940E431F910F91FF900895EF92A1
:106F9000FF920F931F93BC018FE199E00E94493546
:106FA0000AE613E038E0F32EF0926A0310926B03C6
:106FB000C80102966AE37EE049E050E00E94320890
:106FC00084E580936F03EE24E394E09275030E94BE
:106FD0000035F09280031092810310928203109288
:106FE000830385E080938403809154098093850313
:106FF00010928603E0928703C8014E9662E470E027
:1070000048E350E00E94480884E262E240E450E035
:1070100020E00E94943482E690E00E940E431F918B
:107020000F91FF90EF900895DF92EF92FF920F93F0
:107030001F93CF93DF93EC0180916909882319F0A6
:10704000CE010E94683F209709F0BFC080911409CB
:107050008570F1F18091C9029091CA02892BC1F526
:107060000E9446428823A1F184E293E00E943835D1
:1070700088E080936A03A6E0FA2EF0926B038CE618
:1070800093E062E37EE048E050E00E9432080EE7C1
:1070900013E0D8011D92FA94E9F7C8010A976BE44E
:1070A00079E00E949C41C801069669E579E00E945A
:1070B000A441C801049761E579E00E94A441809150
:1070C00014098860809314098AE290E00E940E43BC
:1070D0008091C9029091CA0201969093CA0280934E
:1070E000C90280911509813009F002C2809114090A
:1070F00081FFFEC102E0009315098091CB028F5FF2
:107100008093CB028F71109116091295110F107E8A
:10711000182BE0901709D09018098FE199E065E6E7
:1071200079E00E944935F8E0FF2EF0926A03109250
:107130006B038CE693E06AE37EE049E050E00E9456
:1071400032088CE280936F0386E0809375030E947F
:107150000035E0928203D09283038BE0809380031A
:1071600010938103E4E8F3E0DF011D92FA94E9F75C
:107170008091CC02809386038D5F8093CC0280E661
:1071800080938C0300938D0383E080938E03109291
:107190008F03109290031092910310929203109219
:1071A00093030093940384E08093950300939603E4
:1071B00086E28093970382E36AE140E250E022E0B6
:1071C0000E9494348AE390E0AEC080917C038F3EAD
:1071D00079F480917D038F3F59F480917E038F3F36
:1071E00039F480917F038A3F19F42AE230E082C1AA
:1071F000C932D10508F47CC110916A03183009F036
:1072000082C180916B03863009F07DC184E893E0F0
:1072100061E579E044E050E00E943B08009709F006
:1072200072C180917303813029F584E693E00E9456
:1072300038351092720382E0809373038EE793E0F7
:1072400064E773E00E949C4184E793E06BE479E09B
:107250000E949C4184E893E06AE773E00E94A441A5
:107260008AE793E061E579E00E94A4418AE290E038
:107270000E940E438091140983FF3AC11091730359
:10728000123009F035C18AE793E069E579E044E01E
:1072900050E00E943B08009709F02AC18FE199E075
:1072A00064E773E00E949C411093140921C11830D7
:1072B00009F01EC180916B03882309F019C18091E8
:1072C0006C03853409F014C18CE793E061E579E043
:1072D00044E050E00E943B08009709F009C180910A
:1072E0007503813019F5809180038830F9F4E091BD
:1072F0001909F0911A09309719F088E793E0099578
:107300000E94A8351092800380918203883F28F064
:10731000809183038F5F8093830380918203885FD2
:1073200080938203CE010E940E43E2C00E942F3E52
:10733000882351F080917503813131F4CE010E9490
:10734000343E882309F0D4C0C633D10528F4809197
:107350007503863009F0CCC0809182038B3009F030
:10736000BEC088E793E065E679E044E050E00E9423
:107370003B08009709F0BCC080918D03382F82FF35
:1073800013C0E0911B09F0911C09309759F08091CE
:10739000830382958695877063E040E050E020E0AB
:1073A00030E0099585E090C090916E0380E02091D7
:1073B0006F03022F10E0082B192B80918C03482FAC
:1073C00050E0E4E055954795EA95E1F7CA01880F4A
:1073D000991F880F991F081B190B0451104017FFA4
:1073E00002C000E010E080911509823079F531FF8C
:1073F00021C034FF1FC080E090E060E00E9428368A
:1074000088E180938D03E0911D09F0911E0930976A
:1074100019F420E030E007C08091810382958695C1
:10742000877009959C0183E080931509C9010E942A
:10743000D0355EC081E08093150934FF03C080E041
:1074400090E002C0C801019664E046C0833081F537
:107450000115110579F1E0911B09F0911C09309794
:1074600049F1440F551F440F551FCE0108974E5D3B
:107470005F4F8417950708F4AC01C801840F951F6E
:10748000C817D90710F0980103C09E01241B350BC3
:107490008091830382958695877060E0099580913D
:1074A0006A09882319F0C80168E016C0C80108C03D
:1074B0008530F1F030FF0BC08330D1F0C801019668
:1074C00069E00E94283686E08093150911C00115F5
:1074D000110571F0C80160E00E94283609C0809152
:1074E000CD029091CE02BE010E94A5369C0102C041
:1074F00020E030E0C901DF91CF911F910F91FF9003
:10750000EF90DF900895CA32D10508F0D0CEF0CFC9
:10751000BC01809175038130A1F4809180038823A0
:1075200081F480918803823461F488E793E044E039
:1075300050E00E943B089C0180E0232B19F481E07D
:10754000089580E008950F931F93CF93DF939C01DC
:10755000EB018A0110926909009729F081E599E011
:10756000B9010E94A441209719F0CE010E94C735AD
:107570000115110529F081E699E0B8010E94A441A6
:1075800081E0DF91CF911F910F910895AF92BF924B
:10759000CF92DF92FF920F931F93CF93DF938C01D3
:1075A000EB01F42E1092690938E341E050E060E00D
:1075B00070E018C0832F90E0FC01B3E0F595E795EB
:1075C000BA95E1F7E55DF64F877090705A016B014F
:1075D00004C0AA0CBB1CCC1CDD1C8A95D2F72081F0
:1075E0002A292083315031F78BE499E0BE010E94B3
:1075F0009C41C8016BE479E04F2D0E946A43DF9102
:10760000CF911F910F91FF90DF90CF90BF90AF90DF
:107610000895CF92DF92EF92FF920F931F93DF9323
:10762000CF93CDB7DEB7EB84FC84CD84DE84DE015E
:107630001F9601C0D801F6018491882309F4BCC0CB
:107640000894C11CD11C843209F099C0F601089439
:10765000C11CD11C8491863409F45FC0873434F492
:10766000843469F0853409F08AC06EC08C34C9F165
:10767000833509F445C0883409F081C00DC08D01FF
:107680000E5F1F4FF701668177818D919C914AE0D3
:1076900050E00E94F1087EC02C91822F992787FD2F
:1076A000909514E0959587951A95E1F78F702F7056
:1076B0002A300CF0295F8A300CF0895F8D010E5F53
:1076C0001F4FF701A681B781805DFD018193205D89
:1076D00011962C933196D7011796FC93EE9316973B
:1076E000A9CF8D010C5F1F4F6D917D918D919C9164
:1076F000F701468157812AE030E00E942F094AC0F5
:107700008D010E5F1F4F6D917C91D70116968D9163
:107710009C9117970E9458083DC08D010E5F1F4F26
:107720002D913C910AC0D7011696ED91FC911797C7
:1077300081931796FC93EE931697F9012F5F3F4FB5
:107740008491882381F776CF8D010E5F1F4F2D9195
:107750003C910AC0D7011696ED91FC911797819341
:107760001796FC93EE931697F999FECF32BD21BD83
:10777000F89A80B52F5F3F4F882361F75BCFF70101
:1077800026813781F90181939F01F7013783268391
:107790008D0150CFD70116968D919C911797FC01C2
:1077A00001900020E9F73197E81BF90B8E0F9F1F1E
:1077B000F701978386833ECFCF91DF911F910F9181
:1077C000FF90EF90DF90CF90089580936B0908951C
:1077D0001F93CF93DF930E949A51EB011FEF09C0D3
:1077E0000E949A516C1B7D0B6955724010F08FE01E
:1077F0000CC01EBD0DB407FEFDCF8EB58F3F81F3CB
:107800008E3F11F481E00DC08DE080936D09E09111
:107810006E09F0916F09808190917009892B8083A6
:1078200080E0DF91CF911F910895FF920F931F93F6
:10783000CF93DF938C010E949A51EB01FF24FA94BD
:10784000FEBC0DB407FEFDCF8EB58F3F11F481E075
:1078500008C00E949A516C1B7D0B6017710780F362
:1078600080E0DF91CF911F910F91FF900895DF92FB
:10787000EF92FF920F931F93182FD42EE52EF62E22
:10788000072FE0916E09F0916F0990818091700946
:107890008095892380838CE291E00E94153C812FA2
:1078A00080648EBD0DB407FEFDCF0EBD0DB407FE86
:1078B000FDCFFEBC0DB407FEFDCFEEBC0DB407FE40
:1078C000FDCFDEBC0DB407FEFDCF112311F485E919
:1078D00005C0183011F487E801C08FEF8EBD0DB4DC
:1078E00007FEFDCF90E02FEF2EBD0DB407FEFDCFBC
:1078F0008EB587FF02C09150B9F71F910F91FF908D
:10790000EF90DF900895EF92FF920F931F93CF9324
:10791000DF93EC017A018B0180916C09833039F09F
:1079200089E0EE0CFF1C001F111F8A95D1F781E141
:10793000B801A7010E94373C8823C9F70E94E83BA1
:10794000882319F410926D091BC08FEF8EBD20E0C3
:1079500030E09FEF0DB407FEFDCF8EB5FE01E20FC4
:10796000F31F80839EBD2F5F3F4F81E02F3F38077D
:1079700089F70DB407FEFDCF8EB5C150DE4F888369
:10798000E0916E09F0916F09808190917009892BC7
:10799000808380E0DF91CF911F910F91FF90EF9056
:1079A0000895DF92EF92FF920F931F93D82E7A01E2
:1079B0008B0187E340E050E060E070E00E94373CDC
:1079C0008D2DB801A7010E94373C1F910F91FF90A8
:1079D000EF90DF900895EF92FF920F931F93CF9354
:1079E000DF93082F0E949A51EB01E0916B098E2FD3
:1079F00090E0FC01E75EF04FE491F0E0EE0FFF1F36
:107A0000EB5FF04F2591349130936F0920936E090D
:107A1000875C904FFC01749170937009E091D102E2
:107A20008E2F90E0FC01E75EF04FE491F0E0EE0F66
:107A3000FF1FEB5FF04FA591B491B0937209A09333
:107A40007109875C904FFC01649160937309E09128
:107A5000D0024E2F50E0FA01E75EF04FE491F0E0E3
:107A6000EE0FFF1FEB5FF04F859194919093750996
:107A700080937409475C504FFA0184918093760992
:107A8000E091D2024E2F50E0FA01E75EF04FE49110
:107A90008E2F90E0880F991F8B5F904FFC01E5902F
:107AA000F490F0927809E0927709475C504FFA0120
:107AB000949190937909F9018081872B8083F70154
:107AC0008081892B80838C91862B8C9380916B098C
:107AD00061E00E94BD528091D00261E00E94BD52DF
:107AE0008091D20261E00E94BD528091D10260E09B
:107AF0000E94BD528091CF0261E00E94BD528091F0
:107B0000CF0261E00E94FC52E0916E09F0916F0992
:107B1000808190917009892B808383E58CBD8DB520
:107B20008E7F8DBD80E02FEF2EBD0DB407FEFDCF03
:107B30008F5F8A30C9F7808190959823908309C020
:107B40000E949A516C1B7D0B615D774010F081E0C3
:107B500048C080E040E050E060E070E00E94373CC8
:107B6000182F813069F788E04AEA51E060E070E060
:107B70000E94373C82FF03C010936C091BC080E059
:107B80002FEF2EBD0DB407FEFDCF9EB58F5F843065
:107B9000C1F79A3A11F082E024C082E080936C0928
:107BA00009C00E949A516C1B7D0B615D774010F0FB
:107BB00088E017C089E240E050E060E070E00E9499
:107BC000D13C882371F780916C09823071F58AE38A
:107BD00040E050E060E070E00E94373C882379F09C
:107BE00086E080936D09E0916E09F0916F098081C4
:107BF00090917009892B808380916D0929C08FEF46
:107C00008EBD0DB407FEFDCF8EB5807C803C19F48F
:107C100083E080936C0980E09FEF9EBD0DB407FE6A
:107C2000FDCF2EB58F5F8330C1F7E0916E09F091E3
:107C30006F09808190917009892B8083073028F02B
:107C400086E180936D0980E003C000650CBD81E092
:107C5000DF91CF911F910F91FF90EF900895809148
:107C6000A209811181E00895CF92DF92EF92FF92F5
:107C70000F931F93CF93DF93CAE7D9E030E0CC2472
:107C8000DD2429C02A814B818091820390E0042F5A
:107C900010E080179107D9F4909183039217B9F4FB
:107CA0008C818823A1F02091850330E0285030405A
:107CB000F0908403EE242E0D3F1DE881F981892F79
:107CC000942F68E773E048E853E0099531E00894A1
:107CD000C11CD11C25968091A20990E0C816D90636
:107CE0008CF2832FDF91CF911F910F91FF90EF9036
:107CF000DF90CF900895DF93CF9300D000D000D0D5
:107D0000CDB7DEB7DE011196EAE2F3E086E001903E
:107D10000D928150E1F786E191E0EEE5F3E0DF01BD
:107D20009C011D9221503040E1F78091A3098330DE
:107D300019F46DE579E003C0BE016F5F7F4F84E405
:107D400090E043E450E00E9461358091A3098330C4
:107D500039F08EE593E0BE016F5F7F4F0E949C413A
:107D600081E0809388038093890386E080938A036F
:107D70008091B0099091B109A091B209B091B30975
:107D800080938C0390938D03A0938E03B0938F0305
:107D90008091A309833039F488E893E00C9661E57B
:107DA00079E00E94A44184EA93E06BE479E00E94C8
:107DB0009C41A4E7B4E0EAEEF2E002C081918D9329
:107DC00032E0E03FF307D1F79091A309992311F036
:107DD00083E001C081E080937A048DE380937B048B
:107DE00087E080937C0481E080937D04AEE7B4E07B
:107DF000EBE4F9E002C081918D9389E0E135F80769
:107E0000D1F78CE08093840480E180938504E3EDD6
:107E1000F2E0A6E8B4E002C081918D9322E0E33E57
:107E2000F207D1F726E934E03093B5092093B4097D
:107E3000913069F582E38093960484E080939704FF
:107E4000D9011296E1E5F9E002C081918D9339E004
:107E5000E535F307D1F786E380939C0484E08093B3
:107E60009D048EE994E09093B5098093B409DC01F8
:107E7000EDE5F9E002C081918D9389E0E136F807E4
:107E8000D1F782EA94E09093B5098093B4092091E8
:107E9000B4093091B509D901E4EEF2E002C0819154
:107EA0008D9382E0EA3EF807D1F7C90106969093D8
:107EB000B5098093B409885893400E9447372696A5
:107EC0000FB6F894DEBF0FBECDBFCF91DF910895FE
:107ED000DF92EF92FF920F931F93CF93DF938C016A
:107EE0008091A309823009F4F7C0833030F48823ED
:107EF00051F1813009F054C14AC0833021F08430FF
:107F000009F04EC1E9C00E949A512091A809309110
:107F1000A9094091AA095091AB09E090A409F090F9
:107F2000A5090091A6091091A7092E0D3F1D401F1C
:107F3000511F621773078407950708F431C10E9427
:107F40007B3E84E017C00E949A516093B009709301
:107F5000B1098093B2099093B3091092510910921C
:107F6000520910925309109254090E947B3E0E94BC
:107F7000154281E08093A3090E949A516093AC0955
:107F80007093AD098093AE099093AF0909C106348F
:107F9000110508F4F0C080918103833409F0EBC02F
:107FA00020918C0330918D0340918E0350918F036B
:107FB0008091B0099091B109A091B209B091B30933
:107FC000281739074A075B0709F0D5C0C8E7D4E08E
:107FD000FE01A801425A5C4FDF01119691819D017B
:107FE0002F5F3F4F8081853321F411968C91823031
:107FF00039F0F901E90FF11DE417F50768F3BBC08B
:1080000081E599E068E973E00E94A4415EE5E52E10
:1080100053E0F52EE00EF11EFE013196D9808F015E
:108020000F5F1F4F88818630A9F0873030F4813090
:1080300059F0833009F045C00AC08633E9F18A332C
:1080400061F08333F1F509C085E599E037C089E532
:1080500099E034C081E699E031C0618170E080E050
:1080600090E0982F872F762F6627F8012181620FE5
:10807000711D811D911D982F872F762F66272281D4
:10808000620F711D811D911D982F872F762F6627F6
:108090002381620F711D811D911D28EE33E040E0A8
:1080A00050E00E9418576093A8097093A909809323
:1080B000AA099093AB0905C08DE599E0B8010E942B
:1080C000A441E801CD0DD11DCE15DF0508F4A4CFE4
:1080D0000E947B3E82E04ECF0634110508F44BC06F
:1080E00080918103833409F046C020918C03309144
:1080F0008D0340918E0350918F038091B009909130
:10810000B109A091B209B091B309281739074A07FC
:108110005B0789F5E8E7F4E0A801425A5C4FDF010C
:10812000119691819D012F5F3F4F8081853321F40E
:1081300011968C91853039F0F901E90FF11DE417A2
:10814000F50768F318C00E9410420E949A5160938C
:10815000A4097093A5098093A6099093A70980911B
:108160005909882321F089E599E00E94C73583E009
:108170008093A30915C00E949A512091AC093091B7
:10818000AD094091AE095091AF09205F384D4F4F76
:108190005F4F261737074807590710F41092A309B5
:1081A000DF91CF911F910F91FF90EF90DF90089595
:1081B000CF93DF9381E08093690990915009892FD3
:1081C00082958F70805D8093E1029F70905D9093A7
:1081D000E2021092A3090E949A51EB0104C00E948E
:1081E00085420E94683F8091A309833061F00E941C
:1081F0009A516C1B7D0B60567A4E28F40E944642C1
:10820000882389F3ECCF90E08091A309833009F4AF
:1082100091E0892FDF91CF910895CF93DF93DC0117
:10822000EB01722F632F822F932F9C01F90150E0F5
:1082300016C08081981771F431968081882371F47B
:1082400011968C918D3331F4872F962F9C01F90173
:1082500051E004C0872F962F9C01F90111969C9143
:10826000992339F0903229F09A3019F0552309F307
:1082700004C0513011F030E018C06A2F50E0415076
:10828000504002C0299311963A2F361B2C9122237D
:1082900059F0203249F02A3039F0263229F0832F64
:1082A00090E08417950774F31882832FDF91CF91A4
:1082B0000895CF93DF93FC01EC0137C08B3211F4AA
:1082C00080E231C0853279F5DF0111969181392F35
:1082D00030533A3070F0892F8156863010F437527F
:1082E00008C0892F8154863010F030E002C0392F49
:1082F0003753FD01319611962C91922F90539A305D
:1083000070F0822F8156863010F4975208C0822F69
:108310008154863010F090E002C0922F9753832F43
:108320008295807F892B899331968081882331F6CD
:108330001882DF91CF910895DC01FB0186E0019066
:108340000D928150E1F708959C01FB01808191819C
:10835000A281B381F90180839183A283B3830895BD
:108360008091B80961E00E94FC5278940895FF92D0
:108370000F931F93082F162FF42EF8948091B809AD
:1083800060E00E94FC521F71102B1EBD0DB407FE51
:10839000FDCFFEBC0DB407FEFDCF0E94B0411F9182
:1083A0000F91FF9008951F93182F282F30E020760B
:1083B00030708091B90990E02817390799F080EA68
:1083C0006FE143E00E94B741412F40764093B909E5
:1083D00050E085E0559547958A95E1F780E86FE193
:1083E0000E94B7411F9108950F931F93182F062FD6
:1083F0000E94D34180E4612F402F0E94B7411F911A
:108400000F9108950F931F93182F072F0E94F44187
:10841000812F8F5F602F0E94F4411F910F9108956B
:1084200088E360EB0E94F441089588E361EB0E94C9
:10843000F44108950F931F93182F062FF8948091FD
:10844000B80960E00E94FC52802F8F71812B8EBD95
:108450000DB407FEFDCF1EBC0DB407FEFDCF07FF18
:1084600004C01EBC0DB407FEFDCF1EB50E94B04176
:10847000812F1F910F9108951F93182F0E94D341B0
:1084800080E0612F0E941A421F91089584ED61E1FE
:108490000E94F44182ED61E00E94F4418AEE0E9464
:1084A0003C4280FDFBCF82ED60E00E94F44189ED0B
:1084B0000E943C4290E096958795969587958170AD
:1084C00008950F931F93CF93DF93EC018B01F894E2
:1084D0008091B80960E00E94FC528AE38EBD0DB421
:1084E00007FEFDCF09C01EBC0DB407FEFDCF8EB543
:1084F000F80181938F0121972097A9F70E94B0413D
:10850000DF91CF911F910F9108950F931F93DF93E8
:10851000CF9300D000D000D0CDB7DEB789E30E9462
:108520003C42882319F400E010E048C06091BA0989
:108530007091BB0980E00E94024286E090E0BE019B
:108540006F5F7F4F0E94614289819A819093BB093E
:108550008093BA092B813C81E091B609F091B7096B
:108560008D8187FD03C000E010E00EC02450304034
:108570008F01015010402017310708F48901C8010C
:108580006EE573E00E946142F801E25AFC4F1082EE
:108590006091BA097091BB098CE06130780724F0D2
:1085A0008CE06FEF7BE003C0615070408CE00E9474
:1085B000024280E86EE140E40E94B741C80126967D
:1085C0000FB6F894DEBF0FBECDBFCF91DF911F91E4
:1085D0000F9108950F931F93CF93DF938C01EB01BD
:1085E000F8948091B80960E00E94FC528AE78EBD41
:1085F0000DB407FEFDCF08C088818EBD0DB407FE07
:10860000FDCF21960150104001151105A9F70E94D8
:10861000B041DF91CF911F910F910895CF93DF93D8
:10862000EC010FC08CE10E943C4281FF0AC080E84F
:108630006FE140E80E94B74180EA6FE140E80E94A4
:10864000B74180E06FE10E941A4283FDEBCF82E0E8
:1086500060E07CE00E940242BE016050744F86E000
:108660000E9402428AE760E040E00E94B741CE01EA
:108670006EE573E00E94EA4280E86FE148E00E9404
:10868000B741DF91CF91089584E061E00E94BD522F
:1086900084E061E00E94FC5285E061E00E94BD52EE
:1086A00087E061E00E94BD5286E060E00E94BD521A
:1086B00085E061E00E94FC5285E060E00E94FC528F
:1086C00087E060E00E94FC5280E58CBD8DB5816042
:1086D0008DBD08951F93CF93DF93EB01142F9093DB
:1086E000B7098093B6090CB406FC02C00E9444434B
:1086F0001093B809812F61E00E94BD520E94B041E1
:108700008FEF60E04FEF0E94B74162E070E080E0E1
:1087100090E00E94A85180E06DE10E941A428823F7
:10872000D1F31092BB091092BA0988E060E070E0C2
:108730000E9402428CE060E070E00E9402428AE007
:108740006FEF7BE00E94024284E060E07CE00E94E8
:10875000024286E06FEF71E10E9402420E941542E0
:1087600088E26FE370E30E94024280E369EF77EFF3
:108770000E94024280EC6DE00E94F44181EC60E0D6
:108780000E94F44180E862EC42E30E94B74186EC2B
:1087900062E17CE00E94024284EC62E10E94F441CA
:1087A0008AEC6CED75E00E94024284EE68810E94C2
:1087B000F44185EE69810E94F44182EE6A810E9453
:1087C000F44183EE6B810E94F44180EE6C810E9443
:1087D000F44181EE6D810E94F44184ED60E10E94DC
:1087E000F44186ED60E071E00E9402428AEE0E9450
:1087F0003C4280FDFBCF8FE10E94D34180E86BE1DA
:1088000040EC0E94B74180E86FE144E00E94B7412C
:1088100082E70E943C42863008F08F5FDF91CF9163
:108820001F9108958F929F92AF92BF92CF92DF9245
:10883000EF92FF920F931F93CF93DF937B018C01F5
:10884000EA012CE330E040E050E00E946A57688380
:10885000C801B7012CE330E040E050E00E946A57C5
:10886000122F032FF42EE52E622F732F842F952FB6
:108870002CE330E040E050E00E946A576983612FAA
:10888000702F8F2D9E2D2CE330E040E050E00E94B1
:108890006A57122F032FF42EE52E622F732F842F89
:1088A000952F28E130E040E050E00E946A576A834B
:1088B000612F702F8F2D9E2D28E130E040E050E099
:1088C0000E946A5779018A01C801B7016C5F7F4F26
:1088D0008F4F9F4F27E030E040E050E00E946A5702
:1088E0006F5F6B8320E0AA24BB24650101C02F5F6A
:1088F000822E9924F401EE54F84FCF0183709070CA
:10890000892B99F4CF0164E670E00E945757892BB8
:1089100039F4CF0160E971E00E945757892B29F49F
:108920008EE691E0A0E0B0E004C08DE691E0A0E02A
:10893000B0E0A80EB91ECA1EDB1EC501A0E0B0E063
:10894000E816F9060A071B0790F62E83F401EE5489
:10895000F84F83E0882E912C8E229F22811491045F
:1089600099F4CF0164E670E00E945757892B39F4DF
:10897000CF0160E971E00E945757892B29F48EE6F8
:1089800091E0A0E0B0E004C08DE691E0A0E0B0E0AE
:10899000A81AB90ACA0ADB0A980187010A191B0931
:1089A0002C093D09CF0164E670E00E9457577C0115
:1089B000CF0160E971E00E945757AC01E0E3F3E0BA
:1089C00060E0613051F48114910449F4E114F10440
:1089D00041F44115510529F002C0808103C08CE1AA
:1089E00001C08DE190E0A0E0B0E0081719072A0768
:1089F0003B0740F0081B190B2A0B3B0B6F5F3196AE
:108A00006C30F9F66F5F6D83802F8F5F8C83DF9101
:108A1000CF911F910F91FF90EF90DF90CF90BF907B
:108A2000AF909F908F900895EF92FF920F931F93B6
:108A30007B018C018091D3099091D409A091D50933
:108A4000B091D609E816F9060A071B0771F0C801AC
:108A5000B70148EC59E00E941244E092D309F09229
:108A6000D4090093D5091093D6091F910F91FF9057
:108A7000EF9008950E9414452091CE0930E02E54C5
:108A8000384FC90108950E9414458091CD0990E0A6
:108A900008950E9414458091CB0990E008950E94AA
:108AA00014458091CC0990E008950E94144580916E
:108AB000C90990E008950E9414458091CA0990E088
:108AC00008954F925F926F927F928F929F92AF9292
:108AD000BF92CF92DF92EF92FF920F931F93CF93AB
:108AE000DF934C01DC0116961C91612F70E080E051
:108AF00090E020E833E341EE51E00E9418575B011B
:108B00006C0122EB37E0E12FF0E0EE54F84F1DC08E
:108B1000C90183709070892BB1F4C90164E670E0DB
:108B20000E945757892B39F4C90160E971E00E940E
:108B30005757892B41F480E891E5A1E0B0E0A80EF9
:108B4000B91ECA1EDB1E2F5F3F4F2E173F0701F7CE
:108B5000D40115968C91482E5524C90164E670E025
:108B60000E9457577C01C90160E971E00E94575784
:108B70008C01C1E0D0E093E0692E712C6222732257
:108B800027C0C230D10591F46114710479F4E11465
:108B9000F10419F40115110549F480E89BE3A6E2FC
:108BA000B0E0A80EB91ECA1EDB1E11C0FE01E15DB9
:108BB000FC4F608170E080E090E020E831E541E02A
:108BC00050E00E941857A60EB71EC81ED91E219647
:108BD000C415D505B4F2D40112966C9170E080E012
:108BE00090E020E13EE040E050E00E9418577B0119
:108BF0008C01F401618170E080E090E02CE330E0D2
:108C000040E050E00E941857E60EF71E081F191F9B
:108C1000D4018C91E80EF11C011D111D14966C916C
:108C200070E061507040882777FD8095982F20E88C
:108C300031E541E050E00E941857E60EF71E081F8C
:108C4000191FEA0CFB1C0C1D1D1DB701C801DF918B
:108C5000CF911F910F91FF90EF90DF90CF90BF9039
:108C6000AF909F908F907F906F905F904F900895FE
:108C70006093F0027093F1028093F2029093F302FA
:108C800008956093BE097093BF098093C0099093C3
:108C9000C1092091F0023091F1024091F20250910D
:108CA000F302260F371F481F591F2093C209309324
:108CB000C3094093C4095093C50982E090E09093A2
:108CC000C7098093C6090E949A516093CF09709397
:108CD000D0098093D1099093D2090895EF92FF9221
:108CE0000F931F931CC02F5F3F4F4F4F5F4F209339
:108CF000BE093093BF094093C0095093C10988EE63
:108D000093E0A0E0B0E0E80EF91E0A1F1B1FE092FE
:108D1000CF09F092D0090093D1091093D2090E9493
:108D20009A51E090CF09F090D0090091D1091091AB
:108D3000D2096E197F09800B910B2091BE093091E9
:108D4000BF094091C0095091C109685E73408040DD
:108D5000904048F68091C2099091C309A091C4093E
:108D6000B091C509281739074A075B07E8F0E09179
:108D7000BC09F091BD093097B9F0099561157105ED
:108D80008105910519F00E9441460EC020E030E0B7
:108D90008091C6099091C709892B11F021E030E03C
:108DA0003093C7092093C6096091BE097091BF092D
:108DB0008091C0099091C1091F910F91FF90EF9090
:108DC00008959093BD098093BC098091BE0990914C
:108DD000BF09A091C009B091C1098093C2099093C5
:108DE000C309A093C409B093C5090E946E460895B3
:108DF000FC01EF5BFD4F1082779610820895109270
:108E0000320C0895FC01E55AFD4F8081882319F446
:108E1000862F0E94E53B0895EF92FF920F931F93D8
:108E20007C018B01472F5527FC01858D968D480FBE
:108E3000591F60E070E0C7018F5B9F4F0E94833C29
:108E40001070000F111F0E0D1F1D0E5B1F4FF8013C
:108E5000308120E08291280F311DC9011F910F91AF
:108E6000FF90EF9008958F929F92AF92BF92CF9212
:108E7000DF92EF92FF920F931F93CF93DF93EC015A
:108E8000C85ADD4F8881C855D240813009F0C4C02E
:108E9000CC5ADD4FE880F9800A811B81C455D2404D
:108EA000E114F1040105110559F4C25BDD4F88811D
:108EB0009981CE54D240892B19F46DEF7FEFB3C066
:108EC000298530E040E050E0C801B7010E946A57B0
:108ED000611571058105910589F4E114F10401051D
:108EE000110561F08E01025B1D4FF80160817181F7
:108EF000CE010E940C47F80191838083A984BB2492
:108F0000CC24DD24EA84FB8400E010E08D899E8976
:108F1000AF89B88DE80EF91E0A1F1B1F6B897C896B
:108F200080E090E02C8530E040E050E00E9418574F
:108F3000E60EF71E081F191FF4E58F2EF2E09F2E94
:108F40008C0E9D1EF4016081718182819381A60146
:108F500095010E946A57E60EF71E081F191F8D859E
:108F60009E85A0E0B0E0E4E0B695A795979587953B
:108F7000EA95D1F7E80EF91E0A1F1B1FC25BDD4FF1
:108F800068817981CE54D24080E090E06250704098
:108F900080409040A60195010E941857E60EF71EEA
:108FA000081F191FCE018F5B9F4FB801A7010E94B8
:108FB000833C882319F0682F70E035C0F4012081CC
:108FC000318142815381DA01C9010196A11DB11D90
:108FD00080839183A283B383C05BDD4FE880F980F7
:108FE0000A811B8179E0880F991FAA1FBB1F7A9500
:108FF000D1F7E816F9060A071B0718F060E072E0DF
:1090000012C069E0220F331F441F551F6A95D1F724
:10901000B701621B730B07C0882319F061EF7FEF64
:1090200002C060EF7FEFCB01DF91CF911F910F91D5
:10903000FF90EF90DF90CF90BF90AF909F908F9078
:1090400008954F925F926F927F928F929F92AF920C
:10905000BF92CF92DF92EF92FF920F931F93CF9325
:10906000DF934C013B018DE390E0880E991EE401F3
:10907000E880F9800A811B81E3ECFFEF8E0E9F1ED2
:1090800049E5442E42E0542E480C591CE2018881E7
:10909000998135E0880F991F3A95E1F7AC01452F8A
:1090A0005527469520E03EEF429FE001439FD00DBB
:1090B000529FD00D1124C80FD91F5A01CC24DD2492
:1090C000AE0CBF1CC01ED11E84010F5B1F4FC80118
:1090D000B601A5010E94833C17C0A096F2018081D1
:1090E0009181019691838083F2E0C030DF0761F4C3
:1090F0000894A11CB11CC11CD11CC801B601A5015A
:109100000E94833CC0E0D0E0F401EC0FFD1FEF5B58
:10911000FF4F8081882309F49DC0DE011B96F40176
:10912000EA0FFB1FEF5BFF4F80818871B1F6F401FE
:10913000EC0FFD1FEF5BFF4F8081853E71F2CF5B2F
:10914000DF4FA4014C0F5D1FC154D04020E030E040
:10915000B301620F731FFA018191AF01FB0180839C
:109160002F5F3F4F2830310599F72896F401EC0F17
:10917000FD1F9E0128503040EF5BFF4F8191E301BE
:10918000898781918A8780818B8718861C86A80DA4
:10919000B91DAF5BBF4F8C918D87280D391D205BAA
:1091A0003F4FF901908180E0E9014A919E01840FCF
:1091B000911DF301978786872D5F3F4FE9019881C5
:1091C00080E0F90142919F01840F911DE301998B89
:1091D000888B255F3F4FF901908180E0E9014A913A
:1091E0009E01840F911DF301938B828B2B5F3F4F68
:1091F000E901488150E060E070E0742F6627552750
:109200004427F901829190E0A0E0B0E0DC019927C9
:109210008827482B592B6A2B7B2BEF019A9180E0F2
:10922000FE01229130E0822B932BA0E0B0E0482B8E
:10923000592B6A2B7B2BF301448B558B668B778BD9
:10924000F401E75AFD4F80819181019691838083DB
:1092500080E001C081E0DF91CF911F910F91FF90DD
:10926000EF90DF90CF90BF90AF909F908F907F90C6
:109270006F905F904F9008956F927F928F929F9220
:10928000AF92BF92CF92DF92EF92FF920F931F9314
:10929000CF93DF93EC016B01ED96E880F9800A81B2
:1092A0001B81ED9789E5A82E82E0B82EAC0EBD1E7D
:1092B000D5011D921C92B1E48B2E912C8C0E9D1E1B
:1092C000C401B801A7010E94833CF4018081882376
:1092D00009F4D8C020E030E022C0205E3F4FD50125
:1092E0008D919C91119701968D939C93B2E02030C3
:1092F0003B0761F40894E11CF11C011D111DC40120
:10930000B801A7010E94833C20E030E0FE01E20F9B
:10931000F31FEF5BFF4F8081882309F4B3C0ABE0FC
:109320006A2E712C620E731EFE01E60DF71DEF5BB7
:10933000FF4F8081887189F6FE01E20FF31FEF5B1A
:10934000FF4F8081853E49F22F5B3F4FBE01620F88
:10935000731F2154304040E050E08601040F151F78
:10936000FB018191BF01D8018C934F5F5F4F483063
:10937000510599F7285F3F4FFE01E20FF31F285078
:109380003040EF5BFF4F8191D60119968C9319976E
:1093900081911A968C931A9780811B968C931B97B8
:1093A00018961C9218971C961C926C0E7D1EE1E478
:1093B000F0E06E0E7F1ED3018C91F60185872C0F95
:1093C0003D1F205B3F4FD9019C9180E0F901429104
:1093D0009F01840F911DD6011F969C938E931E971B
:1093E0002D5F3F4FF901908180E0D9014E919D01A1
:1093F000840F911DF601918B808B255F3F4FD90122
:109400009C9180E0F90142919F01840F911DD6014A
:1094100053969C938E9352972B5F3F4FF901408157
:1094200050E060E070E0742F662755274427D9018B
:109430008E919D0190E0A0E0B0E0DC0199278827A3
:10944000482B592B6A2B7B2BF901929180E02291BA
:1094500030E0822B932BA0E0B0E0482B592B6A2BF5
:109460007B2BD60154964D935D936D937C935797C8
:10947000FE01E75AFD4F808191810196918380839F
:1094800080E001C081E0DF91CF911F910F91FF90AB
:10949000EF90DF90CF90BF90AF909F908F907F9094
:1094A0006F9008956F927F928F929F92AF92BF922A
:1094B000CF92DF92EF92FF920F931F93DF93CF93A0
:1094C000CDB7DEB7A5970FB6F894DEBF0FBECDBF00
:1094D0007C016B01AB0120E030E00CC0FA0190810F
:1094E000892F81568A3108F49052FA019193AF0185
:1094F0002F5F3F4FF60101900020E9F73197EC19FB
:10950000FD092E173F0750F38E01025F1F4FC70161
:10951000B8010E943C49F82EF1E08F1709F490C081
:1095200040E050E0B8019E012F5F3F4F06C0F901B7
:10953000E40FF51F80834F5F5F4FFB01E40FF51FC2
:109540008081803219F04830510589F7CE010196AB
:10955000FC01E40FF51F2EE22083DA01119647E1AA
:10956000642E712C6C0E7D1E8A0F9B1FB301AE0101
:10957000455E5F4F04C0FC012193CF011196FB01B2
:109580002081203229F06F5F7F4F6417750799F7AC
:109590008E010F5F1F4FA00FB11F1C92C801B601B3
:1095A0000E944F080097E9F54DC087ED99E0B5019D
:1095B0000E942148F82E882309F03FC080E090E007
:1095C00005C0F801E80FF91F20830196F501E80FA7
:1095D000F91F2081203219F08830910591F7F801A8
:1095E000E80FF91FE082DC011196C8018A0F9B1F6A
:1095F000A30104C0FC012193CF011196FA0120813F
:10960000203229F04F5F5F4F4815590599F7A00F99
:10961000B11F1C92C801B6010E944F08009729F69D
:1096200011C03EE0A32EB12CAC0EBD1E2EE2E22EE8
:109630009BE1892E912C8C0E9D1EFF2009F4B5CF45
:1096400080E001C081E0A5960FB6F894DEBF0FBEA2
:10965000CDBFCF91DF911F910F91FF90EF90DF90E1
:10966000CF90BF90AF909F908F907F906F90089514
:109670003F924F925F926F927F928F929F92AF92A2
:10968000BF92CF92DF92EF92FF920F931F93DF93DF
:10969000CF93CDB7DEB7A5970FB6F894DEBF0FBE58
:1096A000CDBF8C01B62EC72E342E0F5B1D4FF80197
:1096B000808101541240882311F081E1EFC0862F90
:1096C000972F9C01A90120E030E00CC0FA019081A5
:1096D000892F81568A3108F49052FA019193AF0193
:1096E0002F5F3F4FAB2DBC2DFD0101900020E9F70E
:1096F0003197EA1BFB0B2E173F0740F33EE0E32EAA
:10970000F12CEC0EFD1EC801B7010E943C49D82E79
:10971000F1E08F1709F4C1C040E050E0B7019E01AD
:109720002F5F3F4F06C0F901E40FF51F80834F5FA5
:109730005F4FFB01E40FF51F8081803219F0483044
:10974000510589F7CE010196FC01E40FF51F2EE2C9
:109750002083DA01119627E1422E512C4C0E5D1E1A
:109760008A0F9B1FB201AE01455E5F4F04C0FC0132
:109770002193CF011196FB012081203229F06F5FE8
:109780007F4F6417750799F77E010894E11CF11C5F
:10979000AE0DBF1D1C92C7016B2D7C2D0E944F0882
:1097A000009709F06BC0F701D801AF5BBD4F9E0178
:1097B000225F3F4F81918D93E217F307D9F748C09D
:1097C00087ED99E0B4010E942148D82E882309F042
:1097D00061C080E090E005C0F701E80FF91F208329
:1097E0000196F401E80FF91F2081203219F088302A
:1097F000910591F7F701E80FF91FA082DC0111969E
:10980000C7018A0F9B1FA20104C0FC012193CF0155
:109810001196FA012081203229F04F5F5F4F4615E3
:10982000570599F7AE0DBF1D1C92C7016B2D7C2DFE
:109830000E944F08009721F6F701D801AF5BBD4F9A
:109840009E01225F3F4F81918D93E217F307D9F775
:10985000025B1D4F88A199A1F801819391938AA180
:109860009BA1ACA1BDA181939193A193B1931192BE
:10987000119211921192308280E010C0AEE08A2ED7
:10988000912C8C0E9D1EFEE2AF2EEBE16E2E712C04
:109890006C0E7D1EDD2009F493CF80E1A5960FB6F6
:1098A000F894DEBF0FBECDBFCF91DF911F910F9116
:1098B000FF90EF90DF90CF90BF90AF909F908F90F0
:1098C0007F906F905F904F903F9008950F931F93FC
:1098D000CF93DF93EC01862F0E94EB3C8E010F5B50
:1098E0001F4FC80140E050E060E070E00E94833C00
:1098F000882311F080EF84C1C15CDD4F8881CF5394
:10990000D240853509F079C1C05CDD4F8881C054F3
:10991000D2408A3A09F071C1CD5FDD4F7881C350E2
:10992000D2407883C65FDD4F288130E040E050E0D0
:10993000522F4427332722278A9190E0A0E0B0E0FD
:10994000DC0199278827280F391F4A1F5B1F9A912E
:1099500080E06A91C750D240860F911DA0E0B0E030
:10996000280F391F4A1F5B1F29833A834B835C836F
:10997000C25FDD4F288130E040E050E0522F4427A5
:10998000332722278A9190E0A0E0B0E0DC019927FC
:109990008827280F391F4A1F5B1F9A9180E06A9120
:1099A000CB50D240860F911DA0E0B0E0280F391FA8
:1099B0004A1F5B1F2D833E834F835887743031F0DD
:1099C000763021F0763811F082EF1AC149815A8140
:1099D0006B817C81C8010E94833C882311F080EE5A
:1099E0000FC1C15CDD4F8881CF53D240853509F06E
:1099F00006C1C05CDD4F8881C054D2408A3A09F06C
:109A0000FEC0C25BDF4F8881CE54D0408987C05BE7
:109A1000DF4F988180E02A91CF54D040820F911D72
:109A20009B878A87CF5ADF4F8881C155D0408C876A
:109A3000CD5ADF4F988180E02A91C255D040820FE5
:109A4000911D9E878D87CB5ADF4F988180E02A91A8
:109A5000C455D040820F911DA0E0B0E08F87988B55
:109A6000A98BBA8B0097A105B10531F5CC59DF4F11
:109A7000288130E040E050E0522F4427332722274E
:109A80008A9190E0A0E0B0E0DC0199278827280FB8
:109A9000391F4A1F5B1F9A9180E06A91C156D040DE
:109AA000860F911DA0E0B0E0280F391F4A1F5B1FF1
:109AB0002F87388B498B5A8BC85ADF4F788160E0EB
:109AC0008A91C755D040680F711D7C8B6B8BC05A33
:109AD000DF4F288130E040E050E0522F4427332709
:109AE00022278A9190E0A0E0B0E0DC019927882746
:109AF000280F391F4A1F5B1F9A9180E0EA91CD55CC
:109B0000D0408E0F911DA0E0B0E0280F391F4A1FF2
:109B10005B1F2D8B3E8B4F8B588FC559DF4F288194
:109B200030E040E050E0522F4427332722278A912B
:109B300090E0A0E0B0E0DC0199278827280F391FCA
:109B40004A1F5B1F9A9180E0EA91C856D0408E0F61
:109B5000911DA0E0B0E0280F391F4A1F5B1F298F1D
:109B60003A8F4B8F5C8FEA85FB859F0140E050E088
:109B700089819A81AB81BC81280F391F4A1F5B1FE5
:109B80008C8590E0DC01A69FC001A79F900DB69F39
:109B9000900D1124A0E0B0E0280F391F4A1F5B1F71
:109BA000ED96288339834A835B83ED9789819A8177
:109BB0008E0F9F1F9E8F8D8F860F971F98A38F8F5D
:109BC0006D817E818F81988549E0660F771F881FA0
:109BD000991F4A95D1F70E94275620E030E040E8CF
:109BE00055E30E94B55669A37AA38BA39CA3C55ADB
:109BF000DD4F81E0888380E003C081EF01C081EE0A
:109C0000DF91CF911F910F91089581E08093780C9F
:109C10006093550C1092760C1092770C0895209159
:109C2000540C30E08091530C281B3109C901089570
:109C30004091530C8091540C481718F02FEF3FEFD0
:109C40000AC0E42FF0E0ED5CF34F8081282F30E074
:109C50004F5F4093530CC9010895E091530C8091DC
:109C6000540CE81718F0EFEFFFEF06C0F0E0ED5CE2
:109C7000F34F8081E82FF0E0CF010895089510920E
:109C80007C0C10927B0C88EE93E0A0E0B0E0809317
:109C90007D0C90937E0CA0937F0CB093800C80E49D
:109CA00093E090937A0C8093790C0895CF92DF9291
:109CB000EF92FF920F931F93CF93DF937C016B0181
:109CC0008A018091780C8823A1F0C0E0D0E00DC01B
:109CD000D701ED91FC91D601AC0FBD1F0190F08131
:109CE000E02DC7016C9109952196C017D10780F32B
:109CF00004C0CB01642F0E94884FC801DF91CF912F
:109D00001F910F91FF90EF90DF90CF900895DF9318
:109D1000CF930F92CDB7DEB7FC0169838091780CA9
:109D20008823C9F08091770C803238F081E090E090
:109D30009383828320E030E015C08091760CE82F79
:109D4000F0E0EA5AF34F998190838F5F8093760C0D
:109D50008093770C05C0CE01019661E00E94884F88
:109D600021E030E0C9010F90CF91DF9108950F936A
:109D7000062F8091550C66E57CE04091770C21E040
:109D80000E94334F1092760C1092770C1092780C40
:109D90000F91089561E00E94B74E0895413208F096
:109DA00040E2862F63E37CE00E94EA4E1092530C5F
:109DB0008093540C089521E00E94CE4E0895109295
:109DC000530C1092540C1092760C1092770C0E9447
:109DD00034510895382F413210F040E042C0809154
:109DE000850C8823E1F791E09093850C2093870CF4
:109DF0008FEF8093F20C1092AD0C41504093AE0C5B
:109E00004F5F9093860C8091860C330F832B809349
:109E1000860C8091880C813041F41092880C8091DE
:109E2000860C8093BB0085EC01C085EE8093BC005E
:109E30008091850C8130E1F38091AD0C841710F492
:109E40004091AD0C20E030E00AC0FB01E20FF31FAF
:109E5000D901A357B34F8C9180832F5F3F4F2417B5
:109E6000A0F3842F08950F931F93582F122F413280
:109E700010F081E04AC08091850C8823E1F782E0F0
:109E80008093850C0093870C8FEF8093F20C1092D7
:109E9000AD0C4093AE0CADE8BCE0FB0102C081917B
:109EA0008D938E2F861B8417D0F31092860C809191
:109EB000860C550F852B8093860C8091880C813001
:109EC00041F41092880C8091860C8093BB0085EC45
:109ED00001C085EE8093BC00112321F08091850C98
:109EE0008230E1F38091F20C8F3F11F480E00DC0DD
:109EF0008091F20C803211F482E007C08091F20C64
:109F0000803311F084E001C083E01F910F91089528
:109F1000482F613210F081E008958091850C8430E3
:109F200011F082E008956093D00CAFEABCE0842F7A
:109F30009C01F90102C081918D938E2F841B86179D
:109F4000D0F380E008951F920F920FB60F92112464
:109F50002F933F934F935F936F937F938F939F9331
:109F6000AF93BF93EF93FF938091B90090E0887F08
:109F700090708036910509F4F2C081369105CCF5D8
:109F80008832910509F47BC089329105B4F480319F
:109F9000910509F46FC0813191053CF4009709F4F3
:109FA00047C1089709F04FC165C08831910509F490
:109FB00066C0809709F047C182C08034910509F4DA
:109FC000A4C08134910544F48033910509F482C022
:109FD000C89709F038C189C08035910509F489C056
:109FE0008835910509F496C08834910509F02BC194
:109FF000AEC08839910509F413C189399105ECF493
:10A000008837910509F4ABC0893791054CF488363F
:10A01000910509F4A4C08037910509F014C19FC0CF
:10A020008838910509F4FCC08039910509F49DC078
:10A030008038910509F007C198C0803B910509F46B
:10A04000C6C0813B91054CF4803A910509F49FC04C
:10A05000883A910509F0F7C0BAC0803C910509F42F
:10A06000E3C0883C910509F4DFC0883B910509F005
:10A07000EAC0C2C08091860C8093BB00CFC0909193
:10A08000AD0C8091AE0C981768F49091AD0CE92F4F
:10A09000F0E0E357F34F80818093BB009F5F909384
:10A0A000AD0CBCC08091870C882309F44BC085EDB2
:10A0B0008093BC008091BC0084FDFCCFC2C080E2D4
:10A0C0008093F20C85ED8093BC008091BC0084FDF0
:10A0D000FCCFB7C080E38093F20C85ED8093BC0089
:10A0E0008091BC0084FDFCCFACC088E38093F20C6F
:10A0F0009BC08091AD0C9091BB00E82FF0E0E3573E
:10A10000F34F90838F5F8093AD0C9091AD0C809155
:10A11000AE0C82C08091AD0C9091BB00E82FF0E0B6
:10A12000E357F34F90838F5F8093AD0C8091870C42
:10A13000882341F085ED8093BC008091BC0084FDB4
:10A14000FCCF7FC081E08093880C84EA6EC085EDEF
:10A150008093BC008091BC0084FDFCCF72C083E082
:10A160008093850C1092F10C59C08091F10C8032D3
:10A1700008F056C08091F10C9091BB00E82FF0E000
:10A18000EF52F34F90838F5F8093F10C47C0809123
:10A19000F10C803230F4E091F10CF0E0EF52F34F2B
:10A1A000108285ED8093BC008091BC0084FDFCCFC3
:10A1B0001092850C6091F10CE0918B0CF0918C0C5D
:10A1C00081ED9CE070E009951092F10C2DC084E0C7
:10A1D0008093850C1092CF0C1092D00CE091890CDA
:10A1E000F0918A0C09958091D00C882329F481E0A4
:10A1F0008093D00C1092AF0C9091CF0CE92FF0E02F
:10A20000E155F34F80818093BB009F5F9093CF0C0B
:10A210009091CF0C8091D00C981710F485EC01C070
:10A2200085E88093BC000FC085EC8093BC0009C01A
:10A230001092F20C85ED8093BC008091BC0084FDEF
:10A24000FCCF1092850CFF91EF91BF91AF919F9140
:10A250008F917F916F915F914F913F912F910F90CF
:10A260000FBE0F901F9018951092850C81E080937F
:10A27000870C1092880C81E161E00E94FC5280E121
:10A2800061E00E94FC52E9EBF0E080818E7F8083E8
:10A2900080818D7F808384E38093B80085E4809300
:10A2A000BC0008951F920F920FB60F9211242F93A6
:10A2B0003F938F939F93AF93BF938091F70C9091AF
:10A2C000F80CA091F90CB091FA0C3091FB0C0196AE
:10A2D000A11DB11D232F235D2D3720F02D57019691
:10A2E000A11DB11D2093FB0C8093F70C9093F80CEB
:10A2F000A093F90CB093FA0C8091F30C9091F40CAC
:10A30000A091F50CB091F60C0196A11DB11D8093A2
:10A31000F30C9093F40CA093F50CB093F60CBF9152
:10A32000AF919F918F913F912F910F900FBE0F9002
:10A330001F9018958FB7F8942091F70C3091F80C76
:10A340004091F90C5091FA0C8FBFB901CA010895E0
:10A35000EF92FF920F931F937B018C019FB7F894AC
:10A360002091F30C3091F40C4091F50C5091F60CC7
:10A3700086B5A89B06C08F3F21F02F5F3F4F4F4F00
:10A380005F4F9FBF542F432F322F2227280F311D9D
:10A39000411D511DDA01C90162E0880F991FAA1FF2
:10A3A000BB1F6A95D1F7820F931FA41FB51FBC0175
:10A3B00035C09FB7F8942091F30C3091F40C409184
:10A3C000F50C5091F60C86B5A89B06C08F3F21F086
:10A3D0002F5F3F4F4F4F5F4F9FBF542F432F322F61
:10A3E0002227280F311D411D511DDA01C901E2E06C
:10A3F000880F991FAA1FBB1FEA95D1F7820F931FE1
:10A40000A41FB51F861B970B885E934090F208949B
:10A41000E108F1080109110968517C4FE114F104C8
:10A420000105110531F61F910F91FF90EF900895EE
:10A43000019739F0880F991F880F991F029701978C
:10A44000F1F70895789484B5826084BD84B5816005
:10A4500084BD85B5826085BD85B5816085BDEEE62C
:10A46000F0E0808181608083E1E8F0E0108280810B
:10A4700082608083808181608083E0E8F0E0808179
:10A4800081608083E1EBF0E0808184608083E0EB99
:10A49000F0E0808181608083EAE7F0E08081846081
:10A4A00080838081826080838081816080838081DD
:10A4B000806880831092C10008951F93CF93DF932B
:10A4C000182FEB0161E00E94BD52209709F44AC0A9
:10A4D000CF3FD10509F449C0E12FF0E0E75AF04F32
:10A4E00084918330C1F0843028F4813051F082307F
:10A4F000B1F50CC0863019F1873049F1843079F517
:10A5000014C084B5806884BDC7BD33C084B5806283
:10A5100084BDC8BD2EC0809180008068809380007B
:10A52000D0938900C093880024C08091800080620D
:10A5300080938000D0938B00C0938A001AC08091D2
:10A54000B00080688093B000C093B30012C08091C7
:10A55000B00080628093B000C093B4000AC0C038DD
:10A56000D1051CF4812F60E002C0812F61E00E94C0
:10A57000FC52DF91CF911F910895CF93DF93482F25
:10A5800050E0CA01875C904FFC013491475E504F08
:10A59000FA018491882369F190E0880F991FFC01EA
:10A5A000E550F14FA591B491FC01EB5FF04FC591DF
:10A5B000D491662351F42FB7F8948C91932F9095F2
:10A5C00089238C93888189230BC0623061F42FB773
:10A5D000F8948C91932F909589238C938881832B69
:10A5E00088832FBF06C09FB7F8948C91832B8C93E0
:10A5F0009FBFDF91CF910895482F50E0CA01875A3D
:10A60000904FFC012491CA01875C904FFC0194910A
:10A61000475E504FFA013491332309F440C022239E
:10A6200051F1233071F0243028F42130A1F0223090
:10A6300011F514C02630B1F02730C1F02430D9F420
:10A6400004C0809180008F7703C0809180008F7D4F
:10A650008093800010C084B58F7702C084B58F7D51
:10A6600084BD09C08091B0008F7703C08091B00095
:10A670008F7D8093B000E32FF0E0EE0FFF1FEB5FC4
:10A68000F04FA591B4912FB7F894662321F48C91E3
:10A690009095892302C08C91892B8C932FBF0895AC
:10A6A000682F70E0CB01875A904FFC012491CB01B9
:10A6B000875C904FFC014491675E704FFB01949161
:10A6C000992319F420E030E03CC0222351F12330DB
:10A6D00071F0243028F42130A1F0223011F514C09B
:10A6E0002630B1F02730C1F02430D9F404C0809175
:10A6F00080008F7703C0809180008F7D80938000E1
:10A7000010C084B58F7702C084B58F7D84BD09C029
:10A710008091B0008F7703C08091B0008F7D8093CF
:10A72000B000892F90E0880F991F815F904FFC0146
:10A73000A591B4918C9120E030E0842311F021E0C8
:10A7400030E0C901089508951F920F920FB60F923D
:10A7500011242F933F934F938F939F93EF93FF93E6
:10A760004091C60020913C0D30913D0D2F5F3F4F31
:10A770002F73307080913E0D90913F0D281739074F
:10A7800059F0E0913C0DF0913D0DE450F34F4083C2
:10A7900030933D0D20933C0DFF91EF919F918F9150
:10A7A0004F913F912F910F900FBE0F901F901895D2
:10A7B000E091900DF091910DE05CFF4F81919191AE
:10A7C00020813181821B930B8F739070892B11F044
:10A7D0000E94A35308951F920F920FB60F92112457
:10A7E0002F933F938F939F93EF93FF932091800D2F
:10A7F0003091810D8091820D9091830D281739073A
:10A8000031F48091C1008F7D8093C10014C0E0912C
:10A81000820DF091830DE05CF24F20818091820DDA
:10A820009091830D01968F7390709093830D809318
:10A83000820D2093C600FF91EF919F918F913F91E0
:10A840002F910F900FBE0F901F901895DC011C9652
:10A85000ED91FC911D97E05CFF4F2191319180813A
:10A860009181281B390B2F733070C9010895DC01C9
:10A870001C96ED91FC911D97E05CFF4F208131818A
:10A88000E054F040DF01AE5BBF4F8D919C9111977A
:10A890002817390719F42FEF3FEF07C08D919C91CE
:10A8A000E80FF91F8081282F30E0C9010895DC01ED
:10A8B0001C96ED91FC911D97E05CFF4F208131814A
:10A8C000E054F040DF01AE5BBF4F8D919C9111973A
:10A8D0002817390719F42FEF3FEF10C08D919C9185
:10A8E0001197E80FF91F20818D919C911197019686
:10A8F0008F73907011969C938E9330E0C9010895E8
:10A90000FC0186859785DC01A05CBF4FFC01EE5BF6
:10A91000FF4F2D913C911197808191812817390724
:10A92000C1F70895CF93DF93EC01EE85FF85E05CDE
:10A93000FF4F20813181E054F0402F5F3F4F2F7354
:10A940003070DF01AE5BBF4F8D919C91119728173E
:10A950003907D1F3E05CFF4F80819181E054F040F2
:10A96000E80FF91F6083EE85FF85E05CFF4F3183C0
:10A970002083EE89FF89208181E090E00D8C02C068
:10A98000880F991F0A94E2F7282B208381E090E03A
:10A99000DF91CF9108951092870D1092860D88EE69
:10A9A00093E0A0E0B0E08093880D9093890DA09390
:10A9B0008A0DB0938B0D80E593E09093850D809385
:10A9C000840D8CEF9CE09093910D8093900D80E42A
:10A9D0009DE09093930D8093920D85EC90E0909381
:10A9E000950D8093940D84EC90E09093970D809357
:10A9F000960D80EC90E09093990D8093980D81ECEA
:10AA000090E090939B0D80939A0D86EC90E090934C
:10AA10009D0D80939C0D84E080939E0D83E0809338
:10AA20009F0D87E08093A00D85E08093A10D81E0CC
:10AA30008093A20D0895CF93DF930E9422520E942B
:10AA40007524C8EDD3E50E941C252097E1F30E94F0
:10AA5000D853F9CFCF92DF92EF92FF920F931F93CB
:10AA6000CF93DF937C016B018A01C0E0D0E00FC07F
:10AA7000D6016D916D01D701ED91FC910190F081AE
:10AA8000E02DC7010995C80FD91F015010400115CD
:10AA9000110571F7CE01DF91CF911F910F91FF90BA
:10AAA000EF90DF90CF900895DC01ED91FC91019043
:10AAB000F081E02D09950895CF93DF93DB010D9090
:10AAC0000020E9F71197A61BB70BEC01E881F9818B
:10AAD0000280F381E02DAD010995DF91CF910895BA
:10AAE0004F925F927F928F929F92AF92BF92CF923E
:10AAF000DF92EF92FF920F931F93DF93CF93CDB727
:10AB0000DEB7A1970FB6F894DEBF0FBECDBF2C0104
:10AB1000742ECB01223008F42AE019A231E2C32EB0
:10AB2000D12CCC0EDD1E822E9924AA24BB24672DA5
:10AB3000752FA50194010E946A5779018A01C80105
:10AB4000B701A50194010E941857472D461B089490
:10AB5000C108D1084A3014F4405D01C0495CF601D7
:10AB60004083E114F1040105110521F07E2C5F2DD5
:10AB7000C801DDCFC201B6010E945C55A1960FB697
:10AB8000F894DEBF0FBECDBFCF91DF911F910F9123
:10AB9000FF90EF90DF90CF90BF90AF909F908F90FD
:10ABA0007F905F904F900895CF92DF92EF92FF9247
:10ABB0000F931F93CF93DF93EC016A017B01211563
:10ABC000310541F4E881F9810190F081E02D642F95
:10ABD00009951FC02A303105D1F477FF17C0E881ED
:10ABE000F9810190F081E02D6DE209958C014427F7
:10ABF0005527BA014C195D096E097F09CE012AE07B
:10AC00000E9470559801280F391F04C02AE00E9445
:10AC100070559C01C901DF91CF911F910F91FF9059
:10AC2000EF90DF90CF900895EF92FF920F931F93D4
:10AC30007B019A010027F7FC0095102FB801A701AE
:10AC40000E94D4551F910F91FF90EF900895E894C2
:10AC500009C097FB3EF490958095709561957F4F64
:10AC60008F4F9F4F9923A9F0F92F96E9BB27939512
:10AC7000F695879577956795B795F111F8CFFAF422
:10AC8000BB0F11F460FF1BC06F5F7F4F8F4F9F4F53
:10AC900016C0882311F096E911C0772321F09EE8B1
:10ACA000872F762F05C0662371F096E8862F70E017
:10ACB00060E02AF09A95660F771F881FDAF7880FF1
:10ACC0009695879597F9089597F99F6780E870E0C2
:10ACD00060E008959FEF80EC089500240A94161612
:10ACE000170618060906089500240A94121613067A
:10ACF000140605060895092E0394000C11F4882308
:10AD000052F0BB0F40F4BF2B11F460FF04C06F5F23
:10AD10007F4F8F4F9F4F089557FD9058440F551FF9
:10AD200059F05F3F71F04795880F97FB991F61F0CD
:10AD30009F3F79F087950895121613061406551F44
:10AD4000F2CF4695F1DF08C0161617061806991FB0
:10AD5000F1CF86957105610508940895E894BB27A5
:10AD600066277727CB0197F908950BD0C4CFB5DFBD
:10AD700028F0BADF18F0952309F0A6CFABCF112445
:10AD8000EECFCADFA0F3959FD1F3950F50E0551F8A
:10AD9000629FF001729FBB27F00DB11D639FAA2730
:10ADA000F00DB11DAA1F649F6627B00DA11D661F7F
:10ADB000829F2227B00DA11D621F739FB00DA11DA0
:10ADC000621F839FA00D611D221F749F3327A00D5A
:10ADD000611D231F849F600D211D822F762F6A2FF6
:10ADE00011249F5750408AF0E1F088234AF0EE0F7B
:10ADF000FF1FBB1F661F771F881F91505040A9F788
:10AE00009E3F510570F060CFAACF5F3FECF3983EB4
:10AE1000DCF3869577956795B795F795E7959F5FEE
:10AE2000C1F7FE2B880F911D9695879597F9089588
:10AE3000629FD001739FF001829FE00DF11D649F1E
:10AE4000E00DF11D929FF00D839FF00D749FF00DAA
:10AE5000659FF00D9927729FB00DE11DF91F639F4B
:10AE6000B00DE11DF91FBD01CF0111240895991BFB
:10AE700079E004C0991F961708F0961B881F7A95F1
:10AE8000C9F780950895AA1BBB1B51E107C0AA1FF3
:10AE9000BB1FA617B70710F0A61BB70B881F991F7B
:10AEA0005A95A9F780959095BC01CD01089597FB1F
:10AEB000092E07260AD077FD04D0E5DF06D0002052
:10AEC0001AF4709561957F4F0895F6F790958195E6
:10AED0009F4F0895A1E21A2EAA1BBB1BFD010DC0B6
:10AEE000AA1FBB1FEE1FFF1FA217B307E407F5073A
:10AEF00020F0A21BB30BE40BF50B661F771F881F16
:10AF0000991F1A9469F760957095809590959B01AB
:10AF1000AC01BD01CF010895EE0FFF1F0590F49124
:10AF2000E02D09942F923F924F925F926F927F9201
:10AF30008F929F92AF92BF92CF92DF92EF92FF9249
:10AF40000F931F93CF93DF93CDB7DEB7CA1BDB0BF5
:10AF50000FB6F894DEBF0FBECDBF09942A8839889A
:10AF600048885F846E847D848C849B84AA84B984A1
:10AF7000C884DF80EE80FD800C811B81AA81B981AD
:10AF8000CE0FD11D0FB6F894DEBF0FBECDBFED01C1
:06AF90000895F894FFCFC4
:10AF960074007077006C6F6300747474006E707761
:10AFA60000637077006A7370007069640064006DF6
:10AFB600007900763D5B0072736E00726274006504
:10AFC6006E006D6D00726400743D5B006F70656E9F
:10AFD600646F6F7200426F73746F6E2C4D41006820
:10AFE6007474703A2F2F72617973686F6262792E6A
:10AFF6006E65742F736372697074732F6A617661FC
:10B006002F737663322E302E33000069692D31009E
:10B016007B9101CB219401221F9701C9199A01E660
:10B026001F9D017D20A001921DA3015E0CA6016457
:10B0360016A901640FAF01AE14B2015818B501C5C7
:10B0460013B801E822BB01DD0ABE017D15C1012549
:10B056001BC401480DC701640BCA01F617CB009A41
:10B066000B090B00206CA80B0D0B030101B30B1091
:10B076000B030101BD0B140B01C0FFC70B190B011C
:10B08600A8FFD30B1D0B0101FFDF0B210B0116FFE0
:10B09600EB0B250B01C0FFF70B290B01A8FF040CD6
:10B0A6002D0B0101FF110C310B0101FF1E0C350B9D
:10B0B6000150FF2B0C390B0200FF360C3D0B020131
:10B0C60001370C410B030005470C440B03010158E3
:10B0D6000C480B0300F0690C4C0B030008780C506D
:10B0E6000B03003C880C540B033C78990C590B035A
:10B0F6000001AA0C5E0B030101BB0C620B0364FA90
:10B10600CA0C660B030AF0D80C690B010001E70CA8
:10B116006D0B0300FFF80C720B036EFF030D780B2B
:10B1260001C8FF110D7C0B01CCFF200D800B01091E
:10B13600FF300D850B0136FF400D8A0B0177FF505E
:10B146000D8F0B010001600D940B016B0D6F0D73DC
:10B156000D770D7B0D7F0D830D0100010A50000454
:10B166000506074F70656E537072696E6B6C65727B
:10B176002D3030003703010306FF63825363350128
:10B18600100E00000000000079092A556F0000002B
:10B19600002E6F4F00001F111F11131E00140815FB
:10B1A6000105051500000000CB312A5500004000BE
:10B1B60014005400FFFFFFFFFFFFFFFFFFFFFFFF2D
:10B1C6001F1C1F1E1F1E1F1F1E1F1E1F000000000C
:10B1D600874E564E0F4E184E2D4E3E4E0000000026
:0CB1E60092542A55265457543754805474
:00000001FF
